:100000000C9401120C9400000C9400000C9400005D
:100010000C9400000C9400000C9400000C94F62743
:100020000C9400000C9400000C9451150C940000EA
:100030000C9400000C9400000C9400000C94000040
:100040000C94F1140C9400000C94DD260C94000028
:100050000C94F6260C9400000C9400000C94000004
:100060000C9400000C9400000C9400000C94000010
:100070000C9400000C9400000C941B270C940000BE
:100080000C94B5270C9400000C94000010000001A3
:100090000204081020408000000040008000C000E2
:1000A000000140010500C11100000300D90B000050
:1000B0000300C1110300170E0300D90B0000050057
:1000C000E00800000A00C1110A00170E0A00D90B4F
:1000D0000A00C1110A00170E2800D90B0000000009
:1000E0000000000000000000000000000000000010
:1000F00000000000000000000000000000000700F9
:1001000018C0202020204D904D9040104010489065
:1001100047102020202018C0070000000000070022
:100120001FC03FE03FE0727072707FF07FF0777029
:1001300078F03FE03FE01FC00700000000000780AC
:100140000F100E300C7008F001F003F007F007F00C
:1001500003F001F008F00C700E300F1007001E00C5
:100160008F00C700E300F100F800FC00FE00FE0075
:10017000FC00F800F100E300C7008F001E007E00C5
:1001800081008100810081008100FF0081008100E9
:100190008100FF0081008100810081007E0000005D
:1001A00000000200020007000F801FC03FE03FE098
:1001B0003FE01AC007000F800000000000000000B0
:1001C0000000000000000000000006000F000F000B
:1001D0000600000000000000000000000000FFF02A
:1001E000FFF0FFF0FFF0FFF0FFF0F9F0F0F0F0F0BB
:1001F000F9F0FFF0FFF0FFF0FFF0FFF0FFF000007C
:10020000000000000000060009001080108010802F
:100210001080090006000000000000000000FFF050
:10022000FFF0FFF0FFF0F9F0F6F0EF70EF70EF7015
:10023000EF70F6F0F9F0FFF0FFF0FFF0FFF00000D4
:100240000000000001E000601EA03320618061809A
:10025000618033001E00000000000000000000006C
:10026000000007800CC01860186018600CC0078080
:10027000030003000FC003000300000000000200A1
:100280000300038003C002C002C00280020002001B
:100290000E001E001E000C000000000000000C00FC
:1002A0000E000B0009800CC00E400B4009C038C086
:1002B0007840784031C003C003C0018000000000D6
:1002C0000200020027201FC018C03060707030602C
:1002D00018C01FC02720020002000000000000001C
:1002E0000000100018001C001E001F001F801F00CF
:1002F0001E001C001800100000000000000000009C
:10030000000000800180038007800F801F800F8025
:1003100007800380018000800000000000000000D2
:10032000020007000F801FC002000200020002004E
:1003300002001FC00F800700020000000000000044
:1003400019801980198019801980198019801980E5
:100350001980198000001980198000000000000039
:100360001FE036C066C066C066C036C01EC006C08C
:1003700006C006C006C006C006C00000000000009F
:100380001F8030C0300030001F8030C030C01F8060
:1003900000C000C030C01F8000000000000000004E
:1003A000000000000000000000000000000000004D
:1003B000000000001FE01FE01FE00000000002003E
:1003C00007000F801FC002000200020002000200AE
:1003D00002001FC00F80070002001FC000000000C5
:1003E000020007000F801FC002000200020002008E
:1003F00002000200020002000200000000000000F3
:1004000002000200020002000200020002000200DC
:1004100002001FC00F800700020000000000000063
:100420000000000000000100018001C03FE001C0A9
:10043000018001000000000000000000000000003A
:1004400000000000000004000C001C003FE01C0045
:100450000C0004000000000000000000000000008C
:10046000000000000000000000000000000040004C
:1004700040004000400040007FE00000000000001D
:10048000000000000000088018C038E07FF038E06D
:1004900018C00880000000000000000000000000FC
:1004A0000000000000000000020007000F801FC0D5
:1004B0003FE07FF0000000000000000000000000AE
:1004C00000000000000000007FF03FE01FC00F8030
:1004D0000700020000000000000000000000000013
:1004E000000000000000000000000000000000000C
:1004F00000000000000000000000000000000600F6
:1005000006000F000F000F000F000F00060006008E
:1005100006000000000006000600000000000000C9
:100520000000198019801980198000000000000067
:1005300000000000000000000000000000000000BB
:100540000660066006603FF00CC00CC01980198080
:100550007FC03300330033000000000000000600BD
:1005600006001F803FC0360036003F801FC006C017
:1005700006C03FC01F80060006000000000000000B
:10058000000000103830387038E001C003800700E8
:100590000E001C0038E070E060E000000000000089
:1005A00007000D80198019801B000E001E003E0000
:1005B000336033C031803BC01E60000000000E007D
:1005C0000E000E00060006000C00000000000000F7
:1005D0000000000000000000000000000000038098
:1005E00006000E000C001C001C001C001C001C005F
:1005F0001C000C000E0006000380000000001C0020
:10060000060007000300038003800380038003804B
:1006100003800300070006001C000000000000002B
:100620000000000036C036C01F800F003FC00F0022
:100630001F8036C036C0000000000000000000002F
:100640000000000000000600060006003FC03FC09A
:100650000600060006000000000000000000000088
:10066000000000000000000000000000000000008A
:10067000000000000E000E000E0006000C0000003E
:100680000000000000000000000000003FC03FC06C
:10069000000000000000000000000000000000005A
:1006A000000000000000000000000000000000004A
:1006B000000000000E000E000E0000000000000010
:1006C00000100030007000E001C0038007000E0041
:1006D0001C003800700060000000000000000F8067
:1006E0003FE03060607060F061B0633066306C3065
:1006F0007830703030603FE00F8000000000030071
:1007000007001F001F000300030003000300030095
:100710000300030003001FE01FE0000000001FC0F3
:100720003FE070706030607000E001C0038007003F
:100730000E001C0038007FF07FF0000000001FC09A
:100740003FE070706030003000700FE00FC000605C
:100750000030603070703FE01FC00000000001C03A
:1007600003C007C00EC01CC038C070C060C07FF09E
:100770007FF000C000C000C000C0000000007FF09B
:100780007FF06000600060007FC03FE000700030DC
:100790000030603070703FE01FC00000000003C0F8
:1007A00007C00E001C00380030007FC07FE0707072
:1007B0006030603070703FE01FC0000000007FF0CC
:1007C0007FF00060006000C000C001800180030075
:1007D0000300060006000C000C00000000000F8063
:1007E0001FC038E03060306038E01FC03FE07070FC
:1007F0006030603070703FE01FC0000000001FC01C
:100800003FE070706030603070703FF01FF000604B
:1008100000E001C003801F001E0000000000000077
:100820000000000000000E000E000E00000000009E
:1008300000000E000E000E0000000000000000008E
:100840000000000000000E000E000E00000000007E
:1008500000000E000E000E00060006000C0000C096
:1008600001C0038007000E001C00380038001C0087
:100870000E000700038001C000C00000000000005F
:1008800000000000000000003FE03FE0000000002A
:100890003FE03FE0000000000000000000003000EA
:1008A00038001C000E000700038001C001C0038057
:1008B00007000E001C0038003000000000001F8000
:1008C0003FC070E0606060E001C003800700060088
:1008D00006000600000006000600000000001FC021
:1008E0003FE0306067B06FB06DB06DB06DB06DB0AF
:1008F0006FE067C070003FC00FC00000000006003E
:1009000006000F000F000F0019801980198030C0F9
:100910003FC03FC0606060606060000000007F001A
:100920007F8061C060C060C061C07F807FC060E0C8
:100930006060606060E07FC07F80000000000F802A
:100940001FC038E030606000600060006000600040
:100950006000306038E01FC00F80000000007F00A2
:100960007F8061C060C06060606060606060606087
:10097000606060C061C07F807F00000000007FE099
:100980007FE060006000600060007F807F8060002A
:100990006000600060007FE07FE0000000007FE01A
:1009A0007FE060006000600060007F807F8060000A
:1009B00060006000600060006000000000000FC088
:1009C0001FE0386030006000600063E063E060605A
:1009D0006060306038601FE00FE000000000606081
:1009E000606060606060606060607FE07FE06060C9
:1009F00060606060606060606060000000001F8098
:100A00001F8006000600060006000600060006001D
:100A10000600060006001F801F8000000000006026
:100A200000600060006000600060006000600060C6
:100A30006060606070C03FC01F80000000006060A8
:100A400060E061C0638067006E007C007C006E0027
:100A50006700638061C060E06060000000006000CB
:100A60006000600060006000600060006000600086
:100A70006000600060007FE07FE0000000006060D8
:100A800070E070E079E079E06F606F6066606660EA
:100A900060606060606060606060000000006060D6
:100AA0007060706078606C606C60666066606360E7
:100AB000636061E060E060E06060000000000F00E3
:100AC0001F8039C030C060606060606060606060DE
:100AD000606030C039C01F800F00000000007F80C0
:100AE0007FC060E060606060606060E07FC07F80C9
:100AF00060006000600060006000000000000F0007
:100B00001F8039C030C0606060606060606060609D
:100B1000636033C039C01FE00F60000000007F80B9
:100B20007FC060E060606060606060E07FC07F8088
:100B30006700638061C060E06060000000001F80AB
:100B40003FC070E06060600070003F801FC000E048
:100B50000060606070E03FC01F80000000003FC088
:100B60003FC006000600060006000600060006005C
:100B70000600060006000600060000000000606097
:100B80006060606060606060606060606060606065
:100B90006060606030C03FC01F8000000000606087
:100BA0006060606030C030C030C01980198019802A
:100BB0000F000F000F00060006000000000060603C
:100BC0006060606060606060606060606660666019
:100BD0006F6079E070E070E06060000000006060CD
:100BE000606030C030C019800F00060006000F00A2
:100BF000198030C030C0606060600000000060603C
:100C0000606030C030C0198019800F000F000600EE
:100C100006000600060006000600000000007FE057
:100C20007FE000C000C001800300060006000C0049
:100C30001800300030007FE07FE0000000006660B8
:100C400066600F000F000F0019801980198030C0F6
:100C50003FC03FC0606060606060000000006F6087
:100C60005FA039C030C060606060606060606060DC
:100C7000606030C039C01F800F000000000060605D
:100C80006060000060606060606060606060606024
:100C90006060606030C03FC01F80000000001F80A7
:100CA0001F801800180018001800180018001800FD
:100CB0001800180018001F801F80000000000000AE
:100CC0000000000000000000000000000000000024
:100CD000000000000000000000007FF07FF0000036
:100CE00007000700070006000600030000000000E0
:100CF00000000000000000000000000000000000F4
:100D000000000000000000001FC03FE000601FE086
:100D10003FE0606060607FE03FE000000000600056
:100D200060006000600060006F807FC070E0606005
:100D30006060606060E07FC07F80000000000000B5
:100D400000000000000000001F803FC070606000D5
:100D50006000600070603FC01F8000000000006005
:100D600000600060006000601F603FE071E0606054
:100D70006060606070603FE01FE000000000000005
:100D800000000000000000001F803FC070607FE096
:100D90007FC0600070003FC01F800000000007801F
:100DA0000F801C001800180018007F007F0018003A
:100DB00018001800180018001800000000000000BB
:100DC00000000000000000001FE03FE07060606075
:100DD00070E03FE01F60006000E03FC03F806000C7
:100DE00060006000600060006F007F8071C060C0C4
:100DF00060C060C060C060C060C000000000000053
:100E000000000600060000000E000E0006000600AE
:100E10000600060006001F801F8000000000000082
:100E200000000180018000000380038001800180B8
:100E3000018001800180018019801F800F00300037
:100E400030003000300030003180338037003E0009
:100E50003E003700338031C030C0000000000E007B
:100E60000E0006000600060006000600060006004A
:100E70000600060006001F801F8000000000000022
:100E8000000000000000000059807FC07FE0666025
:100E90006660666066606660666000000000000074
:100EA00000000000000000003F803FC030E03060E4
:100EB0003060306030603060306000000000000062
:100EC00000000000000000001F803FC070E0606074
:100ED0006060606070E03FC01F80000000000000A4
:100EE00000000000000000007F807FC060E06060C4
:100EF000606070E07FC06F80600060006000000094
:100F000000000000000000001FE03FE07060606033
:100F1000606070E03FE01F60006000600060000003
:100F2000000000000000000037C03FE038603000E3
:100F300030003000300030003000000000000000C1
:100F400000000000000000003F007F8060007F0084
:100F50003F80018001807F803F0000000000000092
:100F600018001800180018007F007F0018001800F3
:100F70001800180018001F800F80000000000000FB
:100F80000000000000000000606060606060606061
:100F90006060606070E03FE01F60000000000000E3
:100FA00000000000000000006060606030C030C0E1
:100FB000198019800F000F000600000000000000DB
:100FC0000000000000000000666066606660666009
:100FD00066606F603FC039C01080000000000000F4
:100FE000000000000000000060C071C03B801F00D6
:100FF0000E001F003B8071C060C0000000000000B8
:10100000000000000000000030C030C019801980CE
:101010000F000F00060006000C000C001800000076
:1010200000000000000000007FC07F800300060079
:101030000C00180030007FC07FC0000000000000DE
:1010400000006060000000001FC03FE000601FE083
:101050003FE0606060607FE03FE000000000000073
:1010600000006060000000001F803FC070E0606012
:101070006060606070E03FC01F8000000000000002
:1010800000006060000000006060606060606060A0
:101090006060606070E03FE01F60000000000000E2
:1010A0003F007F8060C060C061C0678067C060E053
:1010B0006060606060E067C0678000000000000062
:1010C00000000000000006000F00198030C06060C2
:1010D00060607FE07FE000000000000000000F8003
:1010E0001FC038E030606060600060006000600039
:1010F000306038E01FC00F8006001E001E00000098
:1011000000001980198000006060606060606060AD
:101110006060606070E03FE01F6000000000000061
:1011200001800300060000001F803FC070607FE068
:101130007FE0600070003FC01F80000000000000E2
:1011400006000F00198000001FC03FE000601FE094
:101150003FE0606060607FE03FE000000000000072
:1011600000001980198000001FC03FE000601FE0F0
:101170003FE0606060607FE03FE000000000000052
:101180000C000600030000001FC03FE000601FE0ED
:101190003FE0606060607FE03FE000000000000032
:1011A00006000900060000001FC03FE000601FE0CD
:1011B0003FE0606060607FE03FE000000000000012
:1011C00000000000000000001F803FC070E06000D1
:1011D0006000600070E03FC01F8006001E0000003D
:1011E00006000F00198000001F803FC070607FE084
:1011F0007FE0600060003FC01F8000000000000032
:1012000000001980198000001F803FC070607FE0DF
:101210007FE0600060003FC01F8000000000000011
:101220000C000600030000001F803FC070607FE0DC
:101230007FE0600060003FC01F80000000000000F1
:1012400000001B001B0000000E000E000600060040
:101250000600060006001F801F800000000000003E
:1012600006000F00198000000E000E0006000600A8
:101270000600060006001F801F800000000000001E
:101280000C000600030000000E000E000600060021
:101290000600060006001F801F8000000000198065
:1012A00019800000060006000F000F001980198049
:1012B00030C03FC07FE0606060600000000006005A
:1012C00009000600000006000F000F0019801980B9
:1012D00030C03FC07FE060606060000000000180BF
:1012E000030006007FE07FE0600060007F807F8079
:1012F0006000600060007FE07FE000000000000010
:10130000000000000000000000003DC066600660B4
:101310003FC06600660066603BC00000000007E05A
:1013200007E00F000F001F001B001BC033C033007D
:101330003F007F00630063E063E000000000000006
:1013400006000F00198000001F803FC070E0606041
:101350006060606070E03FC01F800000000000001F
:1013600000001980198000001F803FC070E060609D
:101370006060606070E03FC01F80000000000000FF
:101380000C000600030000001F803FC070E060609A
:101390006060606070E03FC01F80000000000000DF
:1013A00006000F001980000060606060606060608F
:1013B0006060606070E03FE01F60000000000000BF
:1013C0000C00060003000000606060606060606008
:1013D0006060606070E03FE01F600000000000009F
:1013E000000019801980000030C030C019801980B9
:1013F0000F000F00060006000C000C0018001980FA
:10140000198000001F803FC070E060606060606015
:101410006060606070E03FC01F800000000000005E
:10142000000019801980000060606060606060608A
:101430006060606070E03FE01F600000000000003E
:1014400000000000000000001F603FC071E063600A
:1014500066606C6078E03FC06F80000000000000B4
:10146000000007800FC00CC00C000C001F000C0017
:101470000C0018003FE03BC000000000000000002E
:1014800000001F603FC071E063606360666066607B
:101490006C606C6078E03FC06F800000000000006E
:1014A00000000000000030C019800F0006000F008F
:1014B000198030C000000000000000000000038020
:1014C00007C006C006000600060006001F800600D2
:1014D00006000600060036003E001C00000000006A
:1014E000030006000C0000001FC03FE000601FE08A
:1014F0003FE0606060607FE03FE0000000000000CF
:10150000030006000C0000000E000E00060006009E
:101510000600060006001F801F800000000000007B
:10152000030006000C0000001F803FC070E06060F8
:101530006060606070E03FC01F800000000000003D
:10154000030006000C000000606060606060606086
:101550006060606070E03FE01F600000000000001D
:1015600000000EC01B8000003F803FC030E03060B4
:1015700030603060306030603060000000000EC0CD
:101580001B8000006060706078607C606E606760E7
:1015900063E061E060E060606060000000001FC028
:1015A0003FE000603FE07FE060607FE03FE0000000
:1015B0003FC03FC0000000000000000000001F808E
:1015C0003FC070E06060606070E03FC01F8000005E
:1015D0003FC03FC000000000000000000000060007
:1015E000060000000600060006000E001C00380081
:1015F0007060606070E03FC01F800000000000006D
:1016000000001FC03FE070706F306DB06F306DB084
:101610006DB070703FE01FC00000000000000000CF
:1016200000000000FFE0FFE000600060006000607C
:10163000006000000000000000000000000000004A
:1016400000003000700030C031807B0006000DC00B
:10165000186030C0018001E00000000000000000C0
:1016600000003000700030C031807B0006000D604B
:101670001B6033E000600060000000000000060016
:101680000600000000000600060006000F000F0024
:101690000F000F000F000600060000000000000011
:1016A000000000000000000018C03180630031809D
:1016B00018C0000000000000000000000000000052
:1016C00000000000000000006300318018C031807D
:1016D000630000000000000000000000000088809F
:1016E00022208880222088802220888022208880D2
:1016F0002220888022208880222088802220555025
:10170000AAA05550AAA05550AAA05550AAA055501D
:10171000AAA05550AAA05550AAA05550AAA07770CB
:10172000DDD07770DDD07770DDD07770DDD0777069
:10173000DDD07770DDD07770DDD07770DDD006003A
:101740000600060006000600060006000600060069
:101750000600060006000600060006000600060059
:10176000060006000600060006000600FE00FE0059
:10177000060006000600060006000600060003003C
:1017800006000C00060006000F000F0019801980EB
:1017900030C03FC07FE06060606000000000060075
:1017A0000F001980060006000F000F001980198035
:1017B00030C03FC07FE060606060000000000C004F
:1017C00006000300060006000F000F0019801980B4
:1017D00030C03FC07FE0606060600000000000003B
:1017E00000001FC03FE0707067306DB06C306DB0AE
:1017F000673070703FE01FC000000000000036003E
:1018000036003600360036003600F600F6000600D8
:10181000F600F60036003600360036003600360098
:101820003600360036003600360036003600360008
:10183000360036003600360036003600360000002E
:1018400000000000000000000000FE00FE00060096
:10185000F600F60036003600360036003600360058
:1018600036003600360036003600F600F600060078
:10187000FE00FE000000000000000000000000006C
:10188000060006000F801FC03EC03600360036003E
:101890003EC01FC00F800600060000000000606010
:1018A000606030C030C0198019800F000F00060042
:1018B0003FC006003FC00600060000000000000018
:1018C000000000000000000000000000FE00FE001C
:1018D00006000600060006000600060006000600D8
:1018E00006000600060006000600060007F007F0E6
:1018F00000000000000000000000000000000600E2
:10190000060006000600060006000600FFF0FFF0D5
:1019100000000000000000000000000000000000C7
:10192000000000000000000000000000FFF0FFF0D9
:101930000600060006000600060006000600060077
:1019400006000600060006000600060007F007F085
:10195000060006000600060006000600060000005D
:10196000000000000000000000000000FFF0FFF099
:101970000000000000000000000000000000060061
:10198000060006000600060006000600FFF0FFF055
:10199000060006000600060006000600060000001D
:1019A00000000EC01B8000001FC03FE000601FE071
:1019B0003FE0606060607FE03FE0000000000EC03C
:1019C0001B800000060006000F000F001980198020
:1019D00030C03FC07FE06060606000000000360003
:1019E0003600360036003600360037F037F030006B
:1019F0003FF03FF000000000000000000000000089
:101A0000000000000000000000003FF03FF0300048
:101A100037F037F036003600360036003600360034
:101A200036003600360036003600F7F0F7F00000DA
:101A3000FFF0FFF0000000000000000000000000C8
:101A400000000000000000000000FFF0FFF00000B8
:101A5000F7F0F7F036003600360036003600360074
:101A60003600360036003600360037F037F03000EA
:101A700037F037F03600360036003600360000000A
:101A800000000000000000000000FFF0FFF0000078
:101A9000FFF0FFF000000000000000000000360032
:101AA00036003600360036003600F7F0F7F000005A
:101AB000F7F0F7F03600360036003600360000004A
:101AC00060606F603FC070E0606060606060606038
:101AD00070E03FC06F606060000000000000000028
:101AE00000000F001F80188018001C000E00070067
:101AF0000F80198019801F800F00000000003F0038
:101B00003F8031C030C030603060786078603060D5
:101B1000306030C031C03F803F0000000000060050
:101B20000F0019807FE07FE0600060007F807F8091
:101B30006000600060007FE07FE00000000019802E
:101B4000198000007FE07FE0600060007F807F8080
:101B50006000600060007FE07FE00000000018008F
:101B60000C0006007FE07FE0600060007F807F80E7
:101B70006000600060007FE07FE000000000000087
:101B80000600060006000600060006000000000031
:101B900000000000000000000000000000000180C4
:101BA000030006001F801F800600060006000600D6
:101BB0000600060006001F801F80000000000600CF
:101BC0000F0019801F801F80060006000600060017
:101BD0000600060006001F801F800000000019801C
:101BE000198000001F801F80060006000600060006
:101BF0000600060006001F801F800000000006008F
:101C0000060006000600060006000600FE00FE00B4
:101C100000000000000000000000000000000000C4
:101C200000000000000000000000000007F007F0C6
:101C30000600060006000600060006000600FFF08B
:101C4000FFF0FFF0FFF0FFF0FFF0FFF0FFF0FFF01C
:101C5000FFF0FFF0FFF0FFF0FFF0FFF0FFF00000FB
:101C60000000000000000000000000000000FFF085
:101C7000FFF0FFF0FFF0FFF0FFF0FFF0FFF00600D5
:101C8000060006000600060006000000060006002A
:101C9000060006000600060006000000000018000E
:101CA0000C0006001F801F800600060006000600CC
:101CB0000600060006001F801F8000000000FFF0E5
:101CC000FFF0FFF0FFF0FFF0FFF0FFF0FFF000008B
:101CD0000000000000000000000000000000018083
:101CE000030006001F803FC070E0606060606060BD
:101CF0006060606070E03FC01F8000000000000076
:101D00000000000000000F00198030C030C03F808C
:101D100031C030C030C031C03F80300030000600DC
:101D20000F0019801F803FC070E0606060606060DD
:101D30006060606070E03FC01F800000000018001D
:101D40000C0006001F803FC070E060606060606053
:101D50006060606070E03FC01F8000000000000015
:101D600000001D80370000001F803FC070E06060F1
:101D70006060606070E03FC01F80000000000EC027
:101D80001B8000001F803FC070E06060606060608A
:101D90006060606070E03FC01F80000000000000D5
:101DA00000000000000060C060C060C060C060C093
:101DB00071C07FC07EC060006000600060000000F5
:101DC00000003C003C0018001F801FC018C018C055
:101DD0001FC01F8018003C003C00000000003C00B9
:101DE0003C0018001F801FC018C018C018C018C0C1
:101DF0001FC01F8018003C003C0000000000018054
:101E00000300060060606060606060606060606049
:101E10006060606030C03FC01F80000000000600AE
:101E20000F0019806060606060606060606060608A
:101E30006060606030C03FC01F800000000018007C
:101E40000C00060060606060606060606060606000
:101E50006060606030C03FC01F8000000000000074
:101E6000000001800300060030C030C019801980D6
:101E70000F000F00060006000C000C001800018087
:101E800003000600606030C019800F0006000600E5
:101E90000600060006000600060000000000000024
:101EA0000000078007800000000000000000000024
:101EB000000000000000000000000000000003001F
:101EC00006000C0000000000000000000000000000
:101ED0000000000000000000000000000000000002
:101EE000000000000000000000001F801F800000B4
:101EF00000000000000000000000000000000000E2
:101F0000000000000000060006001F801F80060081
:101F1000060000001F801F8000000000000000007D
:101F2000000000000000000000001F801F80000073
:101F30001F801F8000000000000000000000000063
:101F400000007000180030C01980730006000D609A
:101F50001B6033E000600060000000000000000033
:101F60001FE036C066C066C066C036C01EC006C070
:101F700006C006C006C006C006C000000000000083
:101F80001F8030C0300030001F8030C030C01F8044
:101F900000C000C030C01F80000000000000000032
:101FA0000000000000000600060000003FC03FC027
:101FB0000000060006000000000000000000000015
:101FC0000000000000000000000013000F000000EF
:101FD00000000000000000000000000000000F00F2
:101FE0001F80198019801F800F0000000000000072
:101FF00000000000000000000000000000000000E1
:1020000000000000000000000000108039C039C04E
:102010001080000000000000000000000000000030
:1020200000000000000000000000020007000700A0
:102030000200000000000000000000000000180086
:102040003800180018001800000000000000000010
:1020500000000000000000000000000000003C0044
:1020600006001C0006003C0000000000000000000C
:1020700000000000000000000000000000003C0024
:1020800006001C0030003E000000000000000000C0
:102090000000000000000000000000000000000040
:1020A0000000000000000F000F000F000F000F00E5
:1020B0000F00000000000000000000000000000011
:1020C0000000000000000000000000000000000010
:1020D0000000000000000000000000000000000000
:1020E0001E0060077E0700F01EF060F77EF7FBDE43
:1020F0001F00E007FF0700F81FF8E0FFFFFF0000E8
:102100001E0060077E0700F01EF060F77EF7FBDE22
:102110001F00E007FF0700F81FF8E0FFFFFF0300C4
:102120004A0053004A00A3004A00030072007B00EB
:1021300072000300EA0003009A0053009A000300B3
:10214000EA00000040008000C00000014001A00043
:10215000500000000000A000A0005000000000009F
:10216000F8000000FF000000FF0000007F80001E5C
:102170000F80007FE7C0007FFFE0003FFFE0000727
:10218000FFC00001FFC00001FF800001FF0003FF4E
:10219000FE0007FFFC0007FFF00003FFF00003FF55
:1021A000FE00001FFFC001FFFFF001FFFFF801FF6D
:1021B000FFF8007FFFF80007FE00003FFF00007FF0
:1021C000FF80007FFF80007FC100001FE000001F34
:1021D000F000001FF000000FE0000007C000000743
:1021E000C0000007C00000078000000300000003DB
:1021F00000000002000000000000000000000000DD
:10220000E000000000000003900000000000000E4D
:10221000180000000000003808000000000000C0A6
:1022200018000000000003807000000000000C0196
:10223000C00000018006300700000003C00F401CF2
:1022400000000006E01DC0700000000C3039C1C065
:10225000000000181871C7180000001C0CE1DC7C9D
:102260000000000E07C3F1C4000000070386070644
:1022700000000003800E1C0200000001C01C30039F
:1022800000000000E03818010080000070700FC1ED
:1022900083C0000038E003E08E6006001DC000200F
:1022A000FC200F000F8000307030198007000010F4
:1022B000003030C00000001800E06060000000083E
:1022C000038060300000000C0E0030180000000495
:1022D0003800180C00000006E0000C0600000003A7
:1022E00080000603000000000000030180000000E1
:1022F00000000180C0000000000000C0C00000001D
:1023000000000060C000000000000030C0000000BD
:1023100000000030C000000000000030C0000000DD
:1023200000000030C000000000000030C0000000CD
:1023300000000030C000000000000030C0000000BD
:1023400000000030C000000000000030C0000000AD
:1023500000000030E00000000000003070000000CD
:102360000000003018000000000000300C000000E9
:1023700000000030040000000000003FFC000000EE
:102380000000003FFC00436F6C6F72546F75636810
:1023900020567320312E32392000426C6F636B203F
:1023A0000043616C6962726174696F6E004F4B002B
:1023B000253032580025303458002533642E25301E
:1023C000326400253564002564002532640025331D
:1023D0006400444400002564002530325800253153
:1023E0003064004F4E00426C6F636B0077616C6C21
:1023F000610001002D4E414E00000100D70BF22379
:102400000000F894EE27ECBBF1E0F5BFE5BFE093E8
:102410006C00F8E1F1BDE1BD8DE0A2E0BB27ED93DA
:102420008A95E9F780E090E1A0E0B1E0ED930197B3
:10243000E9F7EAEFF3E285919591009761F0A591B4
:10244000B59105901590BF01F00105900D9201978F
:10245000E1F7FB01F0CFEFEFEDBFE0E1EEBFC0E051
:10246000D3E00C94C515E881E03011F01C9A01C04E
:102470001C983CC00E945B2D0E945B2D0E94602D29
:10248000FA93EA93EFE3F0E00E94652D08950E942D
:10249000762A0E94D62A0E946B2D0E945B2D0E94F4
:1024A000712D0E94181AE6E8F3E20E94762DE09161
:1024B0000B03E05DEA930E94101A0E945B2D0E94BC
:1024C0007A2D0E94181AEAE9F3E20E94762D0E9402
:1024D0007F2DEA930E9404170895E881E064E7B92C
:1024E000369A349BFECF349AE4B1F5B12196089523
:1024F000E881F981AA81BB81AE17BF071CF4EA1BF2
:10250000FB0B06C0A881B981EA81FB81EA1BFB0BAA
:102510002496089528970E94AC350E94842DE0935C
:102520008F06F0939006E0919B06F0919C06E09355
:102530008D06F0938E060E94892DE0938B06F09312
:102540008C06E0919906F0919A06E0938906F09343
:102550008A060E948E2DE0E00E94952DA0919B0698
:10256000B0919C06A039E1E0BE07ECF4EFE0E09307
:102570006100E1E00E949D2DE5E00E94A42DE1E0D4
:102580000E94952DEFE0E0936100E8E00E949D2D10
:10259000EAE00E94A42DE0E0EA939FDFE093990631
:1025A000F0939A060AC0E0E0F0E0E0939906F09319
:1025B0009A06E0939B06F0939C060E948E2D0E9443
:1025C000892DA0918B06B0918C06EA0FFB1FA0917C
:1025D0009906B0919A060E94AB2D8F010E94842D1E
:1025E000A0918F06B0919006EA0FFB1FA0919B0669
:1025F000B0919C060E94AB2D9F01E0918B06F0915B
:102600008C060E94B22DFF93EF930E94892D0E94A9
:10261000B22DAF91BF91EA0FFB1FFF93EF93E091B3
:102620009906F0919A060E94B22DAF91BF91EA0FE0
:10263000FB1FE0939506F0939606E0918F06F091CC
:1026400090060E94B82DFF93EF930E94842D0E9464
:10265000B82DAF91BF91EA0FFB1FFF93EF93E0916D
:102660009B06F0919C060E94B82DAF91BF91EA0F96
:10267000FB1FE0939706F0939806A0919506B09102
:102680009606E4E1F0E00E941F330E2EA09197061B
:10269000B0919806E4E1F0E00E941F33E02931F0A8
:1026A000E0E0E887E987EA87EB87B8C00093910606
:1026B0001093920620939306309394060E94BE2DA9
:1026C000989724F40E94C32D98970CF023C0E0E063
:1026D000F0E0E0938106F0938206E0917906F091B4
:1026E0007A06309769F40E94C82D0E94D02D1B975E
:1026F00034F0E1E0F0E00E94D52D0E94DA2D0AC00E
:10270000E230A0E0FA0721F0E330A0E0FA0711F48C
:102710000E9445190E94BE2D999724F00E94C32D56
:1027200099970CF47BC0A1E8B6E00E94E12DA0913E
:102730007906B0917A060E94A63514F00C940E1416
:102740000E94E72D0E94BE2D0E94EC2D0E94F32DC9
:102750000E94F82DE0EFF0E060E070E00E9452335C
:102760007F936F93FF93EF930E94FD2D0F010E94C3
:10277000E72DDF01F001EA1BFB0BAF91BF918F91B9
:102780009F910E941A330E94A2330E94F32D0E944F
:10279000022E0E94C32D0E94EC2DEC83FD836E83DC
:1027A0007F83AC81BD818E819F81E0E4F1E060E0B8
:1027B00070E00E9452337F936F93FF93EF930E94D8
:1027C000072E0F010E94022EDF01F001EA1BFB0B16
:1027D000AF91BF918F919F910E941A330E94A233B3
:1027E000EC83FD836E837F83E885F985E09375062E
:1027F000F0937606EC81FD81E0937706F0937806FE
:10280000E0917506F0917606FA93EA93E0917706E7
:10281000F0917806FA93EA930E94CB180E94B335A0
:102820000C9402170E943F1AE2E0E09301030E9419
:102830000C2E0E940C2E0E94331AE1EAF3E20E9451
:10284000762DE4E1EA930E94A416E0E9F1E00E940B
:10285000112EE4E1EA930E94A4160E94152E0E9414
:10286000A63514F4A895F9CFE2E0E09300030E94A6
:102870005B2D0E941A2E0E94331AEBE10E941F2E3C
:102880000E94152E5F9714F4A895FACF0E94262E69
:10289000A0E0B0E00E942F2EEAE5F0E00E94322E88
:1028A0000E94E72D0E94362E0E94152E5E9714F08E
:1028B000A895FACF0E945B2D0E941A2E0E943A2EF4
:1028C000E2E0E09300030E94412E0E94331AEAE105
:1028D0000E941F2E0E94152E5F9714F4A895FACF20
:1028E0000E94262EA2E0B0E00E942F2EE2E8F0E047
:1028F0000E94322E0E94FD2D0E94362E0E94152E1F
:102900005E9714F0A895FACF0E94412E0E943A2EAD
:102910000E94462E0E945B2D0E94331AE8E10E941D
:102920001F2E0E94152E5F9714F4A895FACF0E94CF
:102930004E2EA4E0B0E00E942F2EEAEAF0E00E94C2
:10294000322E0E94022E0E94362E0E94152E5E9775
:1029500014F0A895FACFE9E6F0E0FA93EA930E9422
:102960005B2D0E943A2E0E94462EEEE1F1E00E947D
:10297000322EE9E10E941F2E0E94152E5F9714F45B
:10298000A895FACF0E944E2EA6E0B0E00E942F2E0E
:10299000E2EDF0E00E94322E0E94072E0E94362EB9
:1029A0000E94152E5E9714F0A895FACFE9E6F0E0A4
:1029B000FA93EA93EEE1F1E0FA93EA930E943A2E59
:1029C0000E940C2EEAEFF0E00E94322EEDEAF3E2D4
:1029D0000E94762DE0EDF7E00E94112E0E943F1A32
:1029E00008950E94572EE4E6E2BF78940E9488186A
:1029F00091DDA0912008A13028F0E0912008E1505D
:102A0000E0932008E0911F08E0931E08E6B3AFEFC3
:102A1000EA27E0931F08E03019F0E3E0E093210893
:102A2000E0911F08A0911E08EA17A9F4A0911F08C1
:102A3000A03021F0A0912008A03069F0A0911F08DB
:102A4000A03041F4A0912008A03021F4A0912108E9
:102A5000A03009F40FC0F894E091FD06E160E09326
:102A6000FD067894E2E3E0932008E0912108E1502C
:102A7000E0932108ACE1B8E00E94E12DE091FE0373
:102A8000EF5FE093FE03A091FE03AE3149F4A09105
:102A9000FD03E3E8EA27E093FD03E0E0E093FE03B3
:102AA00008C00E94572E1A93E6E0E4BD0E94072A50
:102AB0001991E991EFBFF991E991B991A991999192
:102AC000899179916991F9901990099018951A93C3
:102AD000A895C1D1E13011F00C94AC15E091E50658
:102AE000E1501E2FA091E406A13021F40E94652E32
:102AF000E03009F412C00E94652EE093FA06E1E08E
:102B0000E093FD060E946C2EBF010E946C2EE081B6
:102B1000E260DB01EC930E94722EA091E406A230E9
:102B200011F0A430C9F40E94652EE093FB06E5E1A4
:102B3000E093FA06E1E0E093FD060E94652EE030A6
:102B400029F00E946C2EE081E27009F405C01A930E
:102B5000E2E0EA930E94AA1AE091FD03E07889F08E
:102B6000E091FD03EF77E093FD030E94661DE09185
:102B7000FD03E07131F0E091FD03E270EA930E9401
:102B800078190E94092819910895E0E0E5BFE093C3
:102B90006D00E0936C00EBBBEFEFEABBE0E0E8BB5D
:102BA000E7BBE5BBEFEFE4BBE0EFE2BBE1BBE0E39B
:102BB000E3B9ECEBE2B9E0E0E0936200E09361009E
:102BC000EFE0E0936500E0936400E0E0E0BFE7E061
:102BD000E3BFE4E6E2BFE0E0E1BFEFBDEEBDEDBD87
:102BE000ECBDE7BDE6BDEBBDEABDE9BDE8BDE093E8
:102BF0007900E0937800E3E0E5BDE6E0E4BDE0E0E5
:102C0000E3BDE0938B00EAE0E0938A00E0E0E0932C
:102C10008900E0938800E0938100E0938000E2E186
:102C2000E0938700E4E3E0938600E0E0E093850032
:102C3000E0938400E0938300E0938200E0936A00D5
:102C4000E0E3EABFE0E4E9BFE8BFE1E4E7BFE0E0DA
:102C5000E0937D00EBB9E8EDEAB9E6E0E09395009A
:102C6000E0E0E0939000E7E6E9B9E0E0E0939B0064
:102C7000E8EDE0939A00E6E0E0939D00E0E0E09369
:102C80009800E3E3E0939900E0E8E8B9E0E0E0BD14
:102C9000E0E4E7B9E7E8E6B9E0B5EF7EE0BDE0E201
:102CA000E0937000E0E0E0937200E4E4E0937400ED
:102CB000EFE1E1BDEFE0E1BD78940E943F2612D341
:102CC000E1E0EA930E9433120E947F2DE53128F063
:102CD000A8E0B0E0E4E10E9415340E94471221E030
:102CE000E5E1E093FA060E94E72D0F010E94FD2D19
:102CF0000E161F0644F40E94022E0F010E94072E9A
:102D00000E161F060CF08EDDE1E0EA931DD000E008
:102D100010E00436E0E01E0724F40E940928E030A9
:102D200009F005C00E94772E0F5F1F4FF2CF0436C7
:102D3000E0E01E0734F00E94152E5F9714F00E9409
:102D40001214C5DEFECFFFCFE881E03021F4EAEABD
:102D5000F0E00E947A2EA881A13021F4E4EAF0E0AC
:102D60000E947A2EA881A23021F4E0EBF0E00E94CC
:102D70007A2EA881A33021F4EEEBF0E00E947A2EA7
:102D8000A881A43021F4E4ECF0E00E947A2E4EC336
:102D90001A9310E00E947F2EE03031F00E947F2EC7
:102DA000EA933ED31F5FF6CF1881239608951A93B6
:102DB0000A93E0E0E0939D06E0939E0610E0143154
:102DC00090F400E0033068F4A3E01A9FF001EC55A2
:102DD000F94FDF01EE27A00FBE1FE0E2EC930F5F7B
:102DE000F1CF1F5FECCFD4C12A970E94862EE3EC6F
:102DF000F3E2FA93EA93EE85FF850E941A330E946C
:102E00008A2EC6DF2C9608952A970E94862EEAEC19
:102E1000F3E2FA93EA93EE85FF27662777270E946D
:102E20008A2EB6DF2B9608951A930A9300E010E0DD
:102E30000E94912EE03021F00832E0E01E070CF0F5
:102E400007C00E94912EEA93EBD20F5F1F4FF0CF85
:102E50001981088112C3E091E306A091E206EA1706
:102E6000C1F00E94982EAE0FBF1FEC91E093E506D3
:102E70000E94982EEA0FFB1FE181E093E406A091E7
:102E8000E306AF5FEAE00E94A733E093E306E1E0E8
:102E90000895E0E008950E94A02EA981A0830E94D9
:102EA000A02E3196A881A083A091E206AF5FEAE050
:102EB0000E94A733E093E206B1C21A930E94AA2EA1
:102EC000E45FFC4FA0E0A0830E94AA2EEA5EFC4FC4
:102ED000108117FF05C0E12F0E94AF2EA0E0A08354
:102EE00016FF05C0E12F0E94B62EA0E0A0830E942D
:102EF000AA2EEA5EFC4FA0E0A0830E94AA2EEB5E01
:102F0000FC4FA0E0A083188189C2AD970E94AA352A
:102F1000EAADFBADAEADBFADEA0FFB1FAF0110E0F8
:102F2000143188F50E94652EE03041F10E94BD2EDB
:102F3000DF010E94DD33DF01ECADFDADEA17FB07D9
:102F4000E9F40E94C32EDF01EEADFFADAE17BF075F
:102F5000ACF00E94C32E4E175F0784F00E94CC2E67
:102F6000AE0FBF1FEEADFFADAE17BF073CF00E9426
:102F7000CC2EAE0FBF1F4A175B070CF402C01A938A
:102F80009CDF1F5FCDCF10E0143110F00C9482183D
:102F90000E94652EE03011F00C948018ACE01A9F6E
:102FA000F001E45FFC4FAFA90E94DB2EE35FFC4F12
:102FB000AEADBFADA083B1830E94BD2EACADBDADA3
:102FC000A083B183ACE01A9FF001EF5EFC4FAAAD85
:102FD0000E94DB2EEE5EFC4FA8AD0E94DB2EED5E64
:102FE000FC4FA09102030E94DB2EEC5EFC4FA091EF
:102FF0000303A0830E946C2E0F01E091FC03E29575
:10300000E07FA0910403EA0FD001EC930E94E02E30
:10301000A0E00E94DB2EE95EFC4FA0E0A083E0E090
:10302000EE83EDA9FEA9309741F00E94E62EEFA9AC
:10303000F8ADFA93EA930E94062BEBA9FCA930970E
:1030400031F00E94E62EEDA9FEA90E94EB2EE0E0F1
:10305000EEA70E94E62E0E94112B3E2F3B30A8F0D7
:1030600000E00E94EF2E11F00C3008F002C00F5F5C
:10307000F8CF0E94EF2E49F40E94F72E30E00E9414
:10308000E02EDF01E02FE058EC93E0E0E88B3130F8
:10309000F0F000E00E94012F11F00C3008F002C0A7
:1030A0000F5FF8CF0E94012F91F4ABE00A9FF0016F
:1030B000EB5FFB4FFA93EA93FE0138960E94EB2EEA
:1030C00030E00E94E02EDF01E02FE05CEC93313035
:1030D000A8F000E00E94EF2E11F00C3008F002C0C2
:1030E0000F5FF8CF0E94EF2E49F40E94F72E30E0D8
:1030F0000E94E02EDF01E02FE058EC93E12F03C0A7
:103100001F5F42CFEFEF0E94B135EF9621960895F1
:103110001A930A930E94092F3097D1F1E0917B0610
:10312000F0917C06309769F50E94092F0E94E733E1
:10313000E0937B06F0937C06309731F4E0E0F0E01A
:103140000E947A2EE0E01AC00E940E2F0E94092FE2
:103150000E94E733F595E7958F01D801E0E0F1E0B3
:103160000E947833E0938700D801E0E0F1E00E940C
:10317000AA33E09386000E940E2FE0E4E0938B00D8
:1031800007C0ABE7B6E0ED91FD913197FE93EE936A
:103190000991199108951A930A9300E010E01431EF
:1031A00010F00C9411190E94652EE030C1F10E94BC
:1031B000C32EAC81BD81EA17FB0764F50E94BD2ECA
:1031C000DF010E94DD33AA81BB81EA17FB0714F5FA
:1031D000ACE01A9FF001E35FFC4F608171811A9FA0
:1031E000F001EF5EFC4F0E94162FAC81BD81AE173F
:1031F000BF0784F40E94BD2E60817181ACE01A9FEC
:10320000F001EE5EFC4F0E94162FAA81BB81AE1723
:10321000BF070CF004C0E12FEF5F0E2F02C01F5F4D
:10322000BECF003081F0E0918306F0918406A02F9C
:10323000B0E0EA17FB0731F0A0918306B091840655
:10324000109709F401C01FC00E94D02DD29714F42A
:103250000E94C82D0E94D02D1397A1F40A93E1E09B
:10326000EA9319DEE02FF0E0E0938306F093840602
:10327000E02FF0E0E0938706F0938806E2E0F0E0CC
:103280000E94D52D01C001D01DC4E0918306F091AC
:103290008406309701F10E94D02D999734F4E09183
:1032A0008306EA93E2E0EA93F6DD0E94D02D999737
:1032B00034F0E0918306EA93E4E0EA93ECDDE0E0A9
:1032C000F0E00E94D52D0E94DA2DE0E0F0E0E093DE
:1032D0008306F0938406E0E0F0E0E0938706F09345
:1032E00088060895CCD063DDE5E1E093FA06089501
:1032F0000E94AA35A0919F06A43120F4A091A006B7
:10330000A33008F032C0E0919F060E941B2F8F016E
:10331000E091A006F0E0A4E1B0E00E944D339F01EF
:103320000E94212FECE0F0E0FA93EA930E94262F0E
:103330000E940C330E94652DEE81E030B1F0E091E7
:103340009F06A3E0EA9FF001EC55F94FDF01E09101
:10335000A006F0E0AE0FBF1F4C9155270E94212F11
:103360004A93E0E0EA930E94CE260E94B135279668
:1033700008950E94602DA0910703B0910803AE1735
:10338000BF075CF4E0910104F0910204A0910903ED
:10339000B0910A03AE17BF070CF040C0E0910703DD
:1033A000F0910803FA93EA93E0910903F0910A037C
:1033B0000E942A2F0E94CE26A0917D06B0917E0603
:1033C000549734F4A0917F06B091800613970CF0C7
:1033D00012C0E0917D06F0917E06A3E0B0E00E946D
:1033E0002533EC55F94FA0917F06B0918006EA0F86
:1033F000FB1FA981A0830E94312FA0910703B091E8
:1034000008030E94372F0E943B2FE0917D06F09128
:103410007E063196E0937D06F0937E06229608950F
:10342000E881EA93E0910303EA93A3DF21960895EC
:10343000EA81FB81E0937D06F0937E06E881F981C5
:10344000E0937F06F0938006AA81BB81ECE0F0E078
:103450000E944D330E943B2FA881B981E4E1F0E046
:103460000E944D3306C0EA81FB810E943B2FE88118
:10347000F981E0930903F0930A03249608950E94CA
:10348000402F143120F41A9318DD1F5FFACF0E94E9
:103490005B2D0E945B2D0E94602DFA93EA93E091D0
:1034A0000104F09102040E94652D10E01C3048F4E4
:1034B000A9E21A9FF001E757FB4FA0E0A0831F5F2E
:1034C000F5CF10E01C3048F4ABE01A9FF001EB5F41
:1034D000FB4FA0E0A0831F5FF5CFE091FD03EF7EDF
:1034E000E093FD0309C30E94402F143100F50E94B0
:1034F000BD2EDF010E94DD33DF01EB81FC81AE17C1
:10350000BF0784F00E94BD2EDF010E94DD33DF0182
:10351000E981FA81EA17FB072CF00E94E02EE08196
:10352000E03009F402C01A93C8DC1F5FDECF0E94AE
:103530005B2DED81FE81FA93EA930E94602DFA9350
:10354000EA93A985BA850E94482F0E94652D1881AB
:1035500025960895EE970E94AA350E944D2FE030DF
:1035600009F46BC20E944D2FEFAFE07851F00E943A
:10357000E62EFE01EF5BFF4FE0810E94AF2E0E941E
:10358000EB2EEFADE07451F00E94E62EFE01EF5BF2
:10359000FF4FE0810E94B62E0E94EB2E0E94E62E85
:1035A0000E94112BEEAFE0910003E9AFE09101031F
:1035B000E8AF0E946B2D0E94582FE35FFC4F008103
:1035C00011810E94582FE15FFC4F208131810E94C0
:1035D000582FEF5EFC4F408155270E94582FEE5E1A
:1035E000FC4FE081F0E0DE01AE5BBF4FED93FC935A
:1035F0000E94582FEC5EFC4FE081EAAFAAADAF30DD
:1036000011F4E8E0EAAF0E94602FDF010E94262F4C
:103610000E944D330E94652F0E94212F5A934A9396
:103620000E946B2FFA93EA93FE01E35BFF4FE08168
:10363000ACE0EA9FF001ED5EFC4FE081EA930E946E
:1036400076260E94212F0E94722F3A932A930E947D
:10365000782F0E947F2F0E948A2F0E948D2F0E9418
:10366000582FEB5EFC4FE081E07181F00E94212F2A
:103670005A934A930E94712D0E94932FFA01E00FF2
:10368000F11F35970E949A2F0E949F2F0E94582F5A
:10369000EB5EFC4FE081E07269F00E947F2F36976D
:1036A0000E94A72F0E94712D0E94932F0E94212F0C
:1036B0000E949F2F0E94212F1A930A930E948D2F00
:1036C0000E94722F3A932A930E94722F0E948D2F8C
:1036D0000E94AC2FA130B1F41A930A93F9013196EC
:1036E0000E948A2FF9013196FA93EA930E94782F6B
:1036F000F80131960E949A2FF8013196FA93EA93D5
:103700000E948D2F0E94AC2FA230E1F40E947F2FE7
:1037100031970E948A2F0E946B2FE20FF31F31977F
:10372000FA93EA930E94782FFA01E00FF11F319784
:103730000E949A2FFA01E00FF11F3197FA93EA9352
:103740000E948D2F0E94582FEC5EFC4FE081EAAF63
:10375000FE01EC5BFF4FE081E03011F40C94F11CB2
:103760000E94312F0E94B12F0E947833EBAFAEAD93
:10377000EA1710F40C940D1CE1E0E0930103E03033
:1037800041F00E94602FEE0FFF1F34960E94B42F6D
:103790000CF009C0E2E0E09301030E94602FEE0FFD
:1037A000FF1F0E94652FDE01A05CBF4F0D90BC91F2
:1037B000A02D0E94BE2FEA1BFB0BDF010E94C52F2C
:1037C0000E94CA2F32F4FE01E05CFF4F00240192F8
:1037D0000082AEAD0E94D12F0E94B12F0E94D92F3E
:1037E000ECAF0E94AC2FA13021F40E94DC2F0E948C
:1037F000E12F0E94AC2FA23021F40E94DC2F0E9406
:10380000E92FE0E0EFAF0E94EF2FE03029F00E94B7
:10381000EF2F0E94F72FF7CFE4C0FE01E05CFF4FCF
:103820000190F081E02DEE0FFF1FDE01AE5BBF4F78
:103830000D90BC91A02DAE1BBF0BE3E0F0E00E9409
:1038400078330E94CA2F22F4E1E0F0E00E94652F55
:10385000EBADA2E0EA9FF001AEADAE17A8F5E1E056
:10386000E0930103E03041F00E94602F0E9410338A
:1038700036960E94B42F0CF009C0E2E0E0930103F9
:103880000E94602FEE0FFF1F0E94652FEEADEDAF7F
:10389000EDADE150EDAFEDAD0E940030A03219F07A
:1038A000ADADA13008F404C0EDADE150EDAFF3CF04
:1038B000ADAD0E94D12FAE2FFA01B0E0EA17FB07A1
:1038C0003CF3EDADE03011F4EBADEDAFADADECE0C0
:1038D000EA9FF0010E94B12F0E94D92FECAF0E9405
:1038E000AC2FA13021F40E94DC2F0E94E12F0E9416
:1038F000AC2FA23021F40E94DC2F0E94E92FE0E0DF
:10390000EFAFEFAD0E940030A03021F0EDADAFADD4
:10391000AE1708F005C00E94EF2F0E94F72FF1CFDD
:10392000EFAD0E940030A03221F4EEADAFADAE1786
:1039300008F007C0EFADEF5FEFAFEDADEF5FEDAFBC
:10394000EFCFADADEEADEA1BAE2FEBADEA1778F0E1
:10395000ADADEEADEA1BACE0EA9FF001A091000333
:10396000EA9FF0010E94B12F0E94D92F01C0E0E030
:10397000ECAF0E94AC2FA13081F40E94DC2F319675
:10398000FA93EA930E94602F3197DF010E94262F5D
:103990000E94073031960E94322E0E94AC2FA23036
:1039A00071F40E94DC2FFA93EA930E94602F319702
:1039B000DF010E94262F0E9407300E94322EEFADB9
:1039C0000E940030A03039F0ADADEFADEA1BAE2F54
:1039D000EBADEA1708F405C00E94EF2F0E94F72F05
:1039E000EECF0E94582FE95EFC4FE081E030F9F005
:1039F0000E946B2D0E94212F36DDE0E0E09303034F
:103A00000E94582FE95EFC4FE081EA3040F00E94AE
:103A1000582FE95EFC4FE081EA93F6D908C00E9476
:103A2000582FE95EFC4FE081E05DEA93F9DCE9ADF7
:103A3000E0930003E8ADE09301030E94B135EF96F7
:103A4000279608951A930A930091030310E0E894CF
:103A500022F8143148F40E94652EE03011F00E94E3
:103A6000722E1F5FA895F5CF00930303099119915A
:103A700008951A930A930091030310E0143100F59E
:103A80000E94652EE030B1F00E94BD2EDF010E9441
:103A9000DD33DF01EC81FD81EA17FB075CF40E9456
:103AA000BD2EDF010E94DD33DF01EA81FB81AE170D
:103AB000BF070CF002C00E94722E1F5FA895DECFD8
:103AC0000093030319810881269608951A9310E044
:103AD000143190F40E94652EE03029F00E946C2E83
:103AE000E081E17009F406C01A93E091FD03E170F2
:103AF000EA9330DD1F5FECCF199108952C970E9457
:103B0000AA35AD89BE890E94C52FED8BFE8BAB898E
:103B1000BC890E94C52FEB8BFC8BED89FE89A98D9A
:103B2000BA8DEA0FFB1FE98FFA8FEB89FC89AF8909
:103B3000B88DEA0FFB1FEF8BF88FED89FE89AD89F9
:103B4000BE890E941230EE87FF87688B798BEB89E4
:103B5000FC89AB89BC890E941230AE85BF858889FB
:103B600099890E945D35EA87FB876C877D8700E035
:103B700010E0EB89FC89E017F10714F40C94071EA0
:103B8000F8010E941A330E948C34EE83FF83688709
:103B90007987AE81BF81888599850E940F35AA8576
:103BA000BB858C859D850E940F35AE85BF85888934
:103BB00099890E94F0330E94BF340E945534AF01AE
:103BC0005A934A930E943C2D2E2F33270E9419307E
:103BD000E98DFA8DE01BF10B0E942030ED8DFE8DFA
:103BE000E01BF10B0E942A300E941930F801A98DC8
:103BF000BA8DEA0FFB1F0E942030F801AD8DBE8DFB
:103C0000EA0FFB1F0E942A300F5F1F4FB2CF0E94A6
:103C1000B1356B960895EA81F0E0EBBBF5BBF7E1B7
:103C2000F09365001F98E6E1E0936500F09365006E
:103C3000E881F981EBBBF5BBFFE1F0936500EEE1B4
:103C4000E0936500F09365001F9A0C941922E2E25C
:103C5000EBBBE0E0E5BB0C941F220C942A220E94EF
:103C60003030EFE1E0936500E4E6F0E00E94112ED1
:103C7000E5EEEA93E0E0F0E80E943630E0E00E94F2
:103C80003A30E1E0EA93E0E0F1E00E943630E2E031
:103C9000EA93E0E0F4E00E9436300E943E300E9459
:103CA0004330B9DFE8E0EA93E2E0F2E00E94363028
:103CB000E9E0EA930E945B2D0E940B1EEAE0EA9382
:103CC0000E945B2D0E940B1EECE0EA930E945B2D8C
:103CD0000E940B1EEDE0EA930E945B2D0E940B1EDA
:103CE000EFE0EA930E945B2D0E940B1EE0E1EA9355
:103CF0000E945B2D0E940B1EE1E1EA930E947A2D47
:103D00000E940B1EE2E1EA930E945B2D0E940B1EB3
:103D1000E3E1EA930E945B2D0E940B1E0E940C2E91
:103D20000E94F032E0E1EA93E0EBFBE10E943630E2
:103D3000E1E1EA930E947A2D0E940B1E0E940C2E54
:103D40000E94F032E2E1EA93EEE1F1E00E943630C7
:103D50000E940C2E0E94F032E3E1EA93E0E0FFE1E2
:103D60000E943630E9E2EA93EFE1F0E00E9436305B
:103D70000E940C2E0E94F032E0E2EA930E945B2D3A
:103D80000E940B1EE1E2EA930E945B2D0E940B1E33
:103D9000A0910B03A13029F4EBE2EA93ECE0F0E010
:103DA00004C0EBE2EA93E0E2F0E0FA93EA930E94C7
:103DB0000B1EE0E3EA930E945B2D0E940B1EE1E3E1
:103DC000EA930E945B2D0E940B1EE2E3EA930E949D
:103DD0005B2D0E940B1EE5E3EA930E945B2D0E947F
:103DE0000B1EE6E3EA93E1E0F1E00E943630E7E300
:103DF0000E944630E8E30E944630E9E30E944630E4
:103E0000ECE30E944630EDE30E944630E0E5EA93A1
:103E10000E945B2D0E944A30E2E5EA930E945B2DEE
:103E20000E945130A0910B03A13029F4E0E6EA93FF
:103E3000E0E0F7EA04C0E0E6EA93E0E0F7E2FA93B4
:103E4000EA930E940B1EE1E60E943A30EAE6EA930A
:103E50000E945B2D0E940B1EE0E8EA930E945B2DFE
:103E60000E940B1EE1E8EA930E945B2D0E940B1E4C
:103E7000E2E8EA930E945B2D0E940B1EE3E8EA93BE
:103E80000E945B2D0E940B1EE4E8EA930E945B2DCA
:103E90000E940B1EE5E8EA930E945B2D0E940B1E18
:103EA000E0E9EA93E0E1F0E00E943630E2E9EA93EB
:103EB000E0E0F7E00E943630E3E9EA930E947A2DD1
:103EC0000E940B1EE5E9EA93EFE3F3E00E9436302F
:103ED000E7E9EA930E945B2D0E940B1EE8E9EA9352
:103EE0000E945B2D0E940B1EE7E00E943A300E9468
:103EF0000C2E0E94F032E7E0EA93E1E2F0E00E944B
:103F00003630E7E0EA93E3E2F0E00E9436300E94C8
:103F10000C2E0E94F032E7E0EA93E3E7F1E00E9422
:103F2000363008950E945830AE85AA2362F0AD85E0
:103F3000BE85A03FE0E0BE0734F4AB85BC85AF335F
:103F4000E1E0BE070CF04EC00E946630AE0FBF1F0E
:103F5000A03FE0E0BE0714F00E946B300E94743076
:103F6000AE0FBF1FA034E1E0BE0714F00E9479300D
:103F70004985E0E50E948230E1E50E9486300E949A
:103F80008C30E2E50E948F30E3E50E9493300E947E
:103F90008C30E0E20E948230E1E20E948F3057DEF6
:103FA0000BBB15BB2EE13FE100E010E00E94993011
:103FB00064F050E0451730F02093650030936500C1
:103FC0005F5FF8CF0F5F1F4FF1CF47DEE0E5EA9369
:103FD0000E945B2D0E944A30E2E5EA930E945B2D2D
:103FE0000E94513052C00E9458300E946630EA1739
:103FF000FB0729F50E949E3014F40E94A530E3E0EF
:10400000EA93E8E3F0E10E943630E0E20E94823079
:10401000E1E20E948F301BDE0BBB15BB2EE13FE1BE
:104020000B851C850E9499303CF0209365003093ED
:1040300065000F5F1F4FF6CF0E943E3024C00E94E4
:104040007430EA17FB0729F50E94B63014F40E9479
:10405000A530E0E20E948230E1E20E948F300E94AF
:10406000271E0BBB15BB2EE13FE10D851E85E985A3
:10407000FA85E017F1073CF0209365003093650066
:104080000F5F1F4FF4CF0E942D1E0E94B1352F9657
:1040900008950E94BD300E94C430FF93EF930E94A8
:1040A000C8300E94C430AF91BF91EA17FB07D8F126
:1040B0000E949E30ECF420E030E00E94CB30E2170A
:1040C000F307ACF00E94BD300E94D2300E94CB308A
:1040D0000E94D730E1E2EA93EC85FD85E21BF30B09
:1040E0000E9436300E94E1302F5F3F4FE6CF19C06B
:1040F00020E030E00E94C830E217F30794F00E94FD
:10410000BD300E94D2300E94C8300E94D730E1E218
:104110000E94E7300E948C300E94E1302F5F3F4FB9
:10412000E9CF0C940D250E94BD300E94C430FF934E
:10413000EF930E94C8300E94C430AF91BF91EA173C
:10414000FB07E8F50E94B630ECF420E030E00E9476
:10415000EC30E217F307ACF00E94C8300E94D23076
:104160000E94EC300E94F330EE85FF85E21BF30BDA
:104170000E9436300E94FA300E94E1302F5F3F4F9C
:10418000E6CF1BC020E030E00E94BD30E217F3070D
:10419000A4F00E94C8300E94D2300E94BD300E941C
:1041A000F330F901AE85BF850E948C300E94FA3051
:1041B0000E94E1302F5F3F4FE7CF0C940D250C9408
:1041C0000D2525970E94AA35EB850E9400310E949B
:1041D0000C31103110F00C947F2100E0E0910103CC
:1041E0000E1710F00C947721E1E20E948230E0E09B
:1041F000EA87AA85A23010F00C946F210E94183132
:10420000E252FF4F2491203011F40C946A2127FFD1
:1042100050C00E942A31E2E2EBBBE0E0E5BBE7E1FF
:10422000E09365001F98F6E1F0936500E093650068
:10423000EE81EBBBEF81E5BBEFE1FEE1E0936500D2
:10424000F0936500E0936500323080F0F0936500F4
:10425000E0936500333050F0F0936500E093650023
:10426000343020F0F0936500E093650026FF20C015
:10427000F0936500E09365004F5F5F4F3230B0F020
:10428000F0936500E09365004F5F5F4F333070F04F
:10429000F0936500E09365004F5F5F4F343030F07E
:1042A000F0936500E09365004F5F5F4F220FDECF14
:1042B0001F9A220F4F5F5F4F323010F04F5F5F4FFA
:1042C000333010F04F5F5F4F343010F04F5F5F4F6F
:1042D0000C940321EA85EF5FEA870C94F920ED85C1
:1042E000FE853196ED87FE870F5F0C94EE20E88502
:1042F000F9853296E887F9871F5F0C94E9200E94C0
:104300003E300C943B2623970E94AA35E9850E94F3
:1043100000313091000310E0EA851E1710F00C9474
:10432000FB2100E0E09101030E1710F00C94F8213E
:10433000E1E2EA93ED85FE850E943630E0E0E88711
:10434000EB85A885AE1710F00C94F0210E94303157
:10435000203011F40C94EB2127FF34C00E942A3145
:10436000E2E2EBBBE0E0E5BBE7E1E09365001F982C
:10437000F6E1F0936500E0936500EE81EBBBEF8121
:10438000E5BBEFE1FEE1E0936500F0936500E093AB
:10439000650031FF04C0F0936500E093650026FFDF
:1043A00010C0F0936500E093650031FF06C0F09304
:1043B0006500E09365004F5F5F4F220F4F5F5F4FD7
:1043C000EECF1F9A220F31FF02C04F5F5F4F4F5F4A
:1043D0005F4F0C94A821E885EF5FE8870C94A0213B
:1043E000EC85FD853196EC87FD870F5F0C9492215B
:1043F0001F5F0C948C210E943E300C943B26EA8176
:10440000F0E0E5BBFBBBF7E1F09365001F98E6E148
:10441000E0936500F0936500E881F981E5BBFBBBA3
:10442000FFE1F0936500EEE1E0936500F093650035
:104430001F9A23960895E2E2E5BBE0E0EBBBE7E1DB
:10444000E09365001F98E6E1E0936500E7E1E09303
:10445000650008951F9A08950E943030EFE1E093BF
:104460006500E8ECF0E00E94112EE6E4EA93E4EA4D
:10447000F0E00E944531E7E4EA93E3E5F0E00E94D2
:104480004531E8E4EA930E945B2DB9DFE9E4EA9361
:10449000E4E4F0E00E944531EAE40E944931EBE4B3
:1044A000EA93E7E6F0E00E944531ECE4EA93E3E3C7
:1044B000F0E00E944531EDE4EA93E7E7F0E00E9486
:1044C0004531EEE4EA93E2E1F0E00E944531EFE4A9
:1044D000EA93ECE4F0E00E944531E0E5EA93E6E49B
:1044E000F0E00E944531E1E5EA93E4E4F0E00E9467
:1044F0004531E1E0EA930E94712D0E94FF210E9464
:104500004D31E3E2EA93E5E9F0E00E944531E4E26F
:10451000EA93E5E9F0E00E944531E5E2EA93EFEF46
:10452000F0E00E944531E7E20E945231E8E20E9449
:104530005231E9E20E945231EAE20E945231ECE249
:104540000E945231EDE20E945231EAE30E9456315C
:10455000EBE30E945631ECE3EA93E0EFF0E00E94D7
:104560004531EDE3EA930E945B2D0E94FF21E4E1D7
:10457000F0E00E94112EE5E3EA93E8E3F0E00E9408
:104580004531E6E3EA93E8E7F0E00E944531EEE3E7
:10459000EA93E8E3F0E00E944531E0E4EA93EFE0DB
:1045A000F0E00E944531E1E4EA93E0EFF0E00E94A0
:1045B0004531E9E1EA93E9E4F0E00E944531E3E9BD
:1045C000EA93EFE0F0E00E9445310E94772EE0E2AE
:1045D000EA93E0E4F0E00E944531EDE1EA930E94C5
:1045E0007A2D0E94FF21EEE1EA930E945B2D0E944A
:1045F000FF21EFE10E944931E4E4EA93EDE4F0E0C9
:104600000E944531E5E4EA93E1E1F0E00E944531A2
:104610000E94772EECE10E944931E4E1F0E00E9433
:10462000112EEBE1EA93E8E1F0E00E9445310E94AF
:104630005A31EBE1EA93E0E1F0E00E9445310E945B
:104640005A31E3E4EA93E0E8F0E00E944531E4E621
:10465000F0E00E94112EE0E9EA93EFE7F0E00E941B
:104660004531E6E20E9449310E945A31E6E2EA937E
:10467000E4E2F0E00E944531E6E2EA93ECE2F0E0A9
:104680000E9445310E945A31E6E2EA93ECE3F0E001
:104690000E944531E7E50E945231E5E5EA930E9428
:1046A0005B2D0E94FF21EEEFEA93EAE5F0E00E9425
:1046B0004531E7E5EA930E945B2D0E94FF210895B2
:1046C0000E945D31AE85AA2362F0AD85BE85A03F14
:1046D000E0E0BE0734F4AB85BC85AF33E1E0BE0754
:1046E0000CF05DC00E946630AE0FBF1FA03FE0E03F
:1046F000BE0714F00E946B300E947430AE0FBF1FD3
:10470000A034E1E0BE0714F00E94793049850E9490
:104710006B31E3E0EA93EE85FF850E944531E4E0EA
:104720000E9486300E947231E5E00E948630EA0FD6
:10473000FB1F0E9445310E947831E7E0EA93EC8547
:10474000FD850E944531E8E00E9493300E9472315D
:10475000E9E00E949330EA0FFB1F0E9445316BDEB7
:1047600005BB1BBB2EE13FE100E010E00E94993049
:1047700064F050E0451730F02093650030936500F9
:104780005F5FF8CF0F5F1F4FF1CF64DE0E944330B1
:104790000E947F31E8E00E9456310E9486313DC17F
:1047A0000E945D310E946630EA17FB0711F00C94FD
:1047B00025240E949E3014F40E94A530E6E1EA937D
:1047C000E8EEF0E00E944531E4E00E945631E5E079
:1047D000EA93EFE3F1E00E944531E8E0EA930E94BA
:1047E0005B2D0E94FF21E9E0EA93EFEEF0E00E94EA
:1047F0004531E2E0EA93EC85FD850E948B31E3E0F0
:104800000E948E310E9493310E94983114DE05BBC4
:104810001BBB2EE13FE10B851C850E9499303CF0CB
:1048200020936500309365000F5F1F4FF6CF0E9405
:104830002A220E944D310E9443300E947F31E8E0DD
:104840000E9456310E948631E8C00E947430EA17F7
:10485000FB0751F50E94B63014F40E94A5300E9467
:104860006B31E3E0EA93EE85FF85F0700E944531FD
:104870000E947831E7E00E948E310E941B2205BB26
:104880001BBB2EE13FE10D851E85E985FA85E0170A
:10489000F1073CF020936500309365000F5F1F4FD8
:1048A000F4CF0E942A22B9C00E94BD300E94C430B9
:1048B000FF93EF930E94C8300E94C430AF91BF9124
:1048C000EA17FB0710F40C94AF240E949E3034F5D5
:1048D00020E030E00E94CB30E217F307F4F00E94B2
:1048E000BD300E94D2300E94CB300E949E310E9487
:1048F000A831E6E0EA93AC85BD85A21BB30BFD01B0
:104900000E948B31E7E0EA93AC85BD850E94B4310B
:104910000E94BB312F5F3F4FDDCF20C020E030E051
:104920000E94C830E217F307CCF00E94BD300E940D
:10493000D2300E94C8300E949E310E94A831E6E029
:104940000E94E7300E947231E7E00E94E7300E9447
:10495000C1310E94BB312F5F3F4FE2CF5EC00E944A
:10496000BD300E94C430FF93EF930E94C8300E9474
:10497000C430AF91BF91EA17FB0710F00C940D25DE
:104980000E94B63034F520E030E00E94EC30E217AF
:10499000F307F4F00E94C8300E94D2300E94EC303D
:1049A0000E94C831AE85BF85A21BB30BFD010E94DA
:1049B0008B31E3E0EA93AE85BF850E94B4310E945B
:1049C000CF310E94D5310E94BB312F5F3F4FDDCFE9
:1049D00024C020E030E00E94BD30E217F307ECF085
:1049E0000E94C8300E94D2300E94BD300E94C8315F
:1049F000F901AE85BF850E947231E3E0EA93F901C7
:104A0000AE85BF850E94C1310E94CF310E94D53151
:104A10000E94BB312F5F3F4FDECF0E94B1352F96F2
:104A2000089525970E94AA35EB850E94DB310E94EC
:104A30000C31103110F00C94B52500E0E091010329
:104A40000E1710F00C94AD250E9493310E949831FE
:104A5000E0E0EA87AA85A23010F00C94A5250E9418
:104A60001831E252FF4F2491203011F40C94A0250C
:104A700027FF55C0E2E0EA93FA010E948B310E94C1
:104A8000E731E2E2E5BBE0E0EBBBE7E1E0936500A4
:104A90001F98F6E1F0936500E0936500EE81E5BBB9
:104AA000EF81EBBBEFE1FEE1E0936500F093650081
:104AB000E0936500323080F0F0936500E09365008C
:104AC000333050F0F0936500E0936500343020F00F
:104AD000F0936500E093650026FF20C0F093650029
:104AE000E09365004F5F5F4F3230B0F0F0936500A8
:104AF000E09365004F5F5F4F333070F0F0936500D7
:104B0000E09365004F5F5F4F343030F0F093650005
:104B1000E09365004F5F5F4F220FDECF1F9A4F5F1C
:104B20005F4F323050F04F5F5F4F333030F04F5FA8
:104B30005F4F343010F04F5F5F4F220F0C943425DD
:104B4000EA85EF5FEA870C942A25ED85FE8531968C
:104B5000ED87FE870F5F0C941E25E885F985329658
:104B6000E887F9871F5F0C9419250C943B2623973F
:104B70000E94AA35E9850E94DB313091000310E0E4
:104B8000EA851E1710F00C943B2600E0E09101032B
:104B90000E1710F00C943826E6E0EA93ED85FE85BA
:104BA0000E948B31E7E0EA93ED85FE85F0700E946C
:104BB0004531E0E0E887EB85A885AE1710F00C944E
:104BC00030260E943031203011F40C942B2627FF20
:104BD00039C0E2E0EA93FA010E948B310E94E7318A
:104BE000E2E2E5BBE0E0EBBBE7E1E09365001F98A4
:104BF000F6E1F0936500E0936500EE81E5BBEF819F
:104C0000EBBBEFE1FEE1E0936500F0936500E0931C
:104C1000650031FF04C0F0936500E093650026FF56
:104C200010C0F0936500E093650031FF06C0F0937B
:104C30006500E09365004F5F5F4F220F4F5F5F4F4E
:104C4000EECF1F9A220F31FF02C04F5F5F4F4F5FC1
:104C50005F4F0C94E325E885EF5FE8870C94DB2534
:104C6000EC85FD853196EC87FD870F5F0C94C6259A
:104C70001F5F0C94C0250E94B13561960895E1E054
:104C8000E0930B03E8EFFFEFE0932208F093230893
:104C9000E491EF3F39F0E0912208F091230804906D
:104CA00000920B03A0910B03A33019F40E942C2255
:104CB00002C00E942F1EE3E0E0930203E0E0E093D5
:104CC0000303E1E0E0930103E0930003EFEEF0E083
:104CD000E093FF03F0930004EFE3F1E0E0930104BD
:104CE000F0930204E4E1E09306030895A0910B031E
:104CF000A33069F40E94EC310E94EC310E94EC3147
:104D00000E94EC31E885EA930E9460230CC00E9467
:104D1000EC310E94EC310E94EC310E94EC31E885CC
:104D2000EA930E94921F1DC0A0910B03A33069F467
:104D30000E94EC310E94EC310E94EC310E94EC3177
:104D4000E885EA930E94D0230CC00E94EC310E94B7
:104D5000EC310E94EC310E94EC31E885EA930E942C
:104D6000F31F29960895A0910B03A33059F40E94D4
:104D7000F1310E94F131EF81EA93EF81EA930E94D1
:104D8000B7250AC00E94F1310E94F131EF81EA9308
:104D9000EF81EA930E94832128960895A0910B0346
:104DA000A33029F40E94F8310E94112504C00E940A
:104DB000F8310E94E120269608950E94FF311A934F
:104DC0000A931BB10CB1E0919308F0E0EF59F74F53
:104DD0000083A0919308AF5FA0939308A23319F4C6
:104DE000E0E0E093930809911991DAC00E94FF3145
:104DF000E091FA08A091F908EA1751F0A091FF0795
:104E0000A03029F0A0E00A99A1E0A03009F401C087
:104E100011C0E091FA08F0E0EB56F74FE081ECB9F1
:104E2000A091FA08AF5FA093FA08A43619F4E0E065
:104E3000E093FA08B5C0AA93BA93EA93FA93EFB74E
:104E4000EA931A930A9310919B0000919C00E12F22
:104E5000EC7111F00C949127023021F4E1E0E09321
:104E6000930A5FC0E091930AE13029F5E0E0E09316
:104E7000930A0A3229F00E947F2DE05DE017D1F4F9
:104E8000E2E0E093930AE0E0E093940A0E940532A6
:104E9000E550F74FA2E0A0830E940532E0938F0A0D
:104EA000F093900A0E940A32E039A1E0FA0711F467
:104EB0000E940D3236C0E23071F40093940AE3E0B0
:104EC000E093930A0E941432E039A1E0FA0711F44A
:104ED0000E940D3226C0E33021F50E941432E039E1
:104EE000A1E0FA0711F40E940D320330D1F4E0E0A2
:104EF000E093930AA091940AA63529F4E091FD0667
:104F0000E260E093FD06A091940AA33451F4689402
:104F100023F8E0918F0AF091900AE093910AF093C0
:104F2000920A09911991E991EFBFF991E991B9912B
:104F3000A99118951A930E9419320E941E32D9F332
:104F40000E941932E550F74F1081ADE8BAE00E9497
:104F5000E12DE039A1E0FA0731F4E0E0F0E0E09380
:104F60008D0AF0938E0AE12F1FC30E94FF31E0915A
:104F7000960BA091950BEA1781F0E091FC06E030CA
:104F800019F0E89421F808C00E9425320E943332BB
:104F900019F4E0E0E093960B03C0E89420F821F8C0
:104FA000E991EFBFF991E991A9911895E091950BDD
:104FB000F0E0EB56F54FA881A083E091950BEF5FF1
:104FC000E093950B0E94333219F4E0E0E093950BE7
:104FD0000C942A2BE0E0E093960BA091950BA13066
:104FE00020F00E942532689421F80895AA93BA937C
:104FF000EA93EFB7EA93E0E0E093960B0E947F2DEF
:10500000EF5FE093FC06E991EFBFE991B991A991B7
:1050100018952A970E94AA3520E00E9419320E9412
:105020001E3221F0A091970BA23008F02FC023FE72
:105030000AC0E091910AF091920AE0938D0AF093F0
:105040008E0AE89423F876DF1E2F123029F4E1E06F
:10505000E093970BE0E017C0A091970BA130A9F463
:105060000E9438321083133039F4E2E0E093970B5A
:105070000E943832A0E0A083A091980BAC3328F4B2
:10508000E091980BEF5FE093980BC7CFA091970B3F
:10509000A23011F00C94032A21E0E091990BE33443
:1050A00071F4E0919A0BE7703E2F303019F40E94B2
:1050B0003F1A04C00E943E320E94731AA0C1E43419
:1050C00071F4E0919A0BE7703E2F303019F40E9492
:1050D000221D04C00E943E320E94391D90C1E73457
:1050E000B1F5E0919C0BE73469F4A091FA06A53183
:1050F00049F0E0919A0BE053AE2FE0919B0BE05505
:10510000EA1709F023C0E0919A0BE053A8E0B0E061
:105110000E9415340E945B2D0E945B2DEFEEF0E0A3
:105120000E9458320E94652DE0E0E09303030E9444
:105130005B2D0E945B2D0E94181AE6EEF3E20E949E
:10514000762D0E947F2DF0E00E94362E58C1E93462
:1051500031F4E0919A0BE370E093FC0350C1E13429
:10516000E1F4E0919A0BEF70E0930203E0919B0B66
:10517000EF70E0930303E0919C0BEF70E093040366
:10518000E0910303A0910203EA1731F4A091030315
:10519000EFE0EA27E093020332C1EC3439F4E09106
:1051A0009A0BE170EA930E94331229C1E43511F0A1
:1051B0000C944829A0910503A03041F4A0919A0BCA
:1051C000A13320F0A0919A0BAA3308F01EC0E09101
:1051D0009B0BE153A8E9B0E00E945D32E0919A0B8D
:1051E000E1530E2F0E9467320E94E7330E94A72FDF
:1051F0000E94673232960E94E733FA93EA93EAE319
:10520000F0E00E9470320E947632A0910503A13036
:1052100041F4A0919A0BA13320F0A0919A0BA433F2
:1052200008F014C0E0919A0BE153AEE4B1E20E94A1
:105230005D32E0919B0BE153A2E4B1E20E947C322B
:10524000EAE3F0E00E9487320E947632A0910503E3
:10525000A23041F4A0919A0BA13320F0A0919A0BB7
:10526000A43308F014C0E0919A0BE153A8E5B1E231
:105270000E945D32E0919B0BE153A4E5B1E20E94F4
:105280007C32EAE9F0E00E9487320E947632B7C0B1
:10529000E534A1F4E0919A0BE053E0939D06E09190
:1052A0009B0BE153E0939E06E0919C0BE13311F4DC
:1052B000E1E001C0E2E0E0932408A1C0E63459F443
:1052C000A0919A0BA03320F0A0919A0BA33308F081
:1052D00001C095C002C0E63521F4E0E0E0939A0BEE
:1052E0008EC0E83511F00C94F929E0910503E03007
:1052F00031F4E0912408E0930003E1E004C0E1E030
:10530000E0930003E2E0E093010322FC02C00E946C
:105310003A12689422F8A0919E06E4E1EA9FF00117
:10532000A0910103EA9FF001EE5FF0E0EA87FB87BE
:105330000E94312FF0E0E887F987E0910103A4E1B2
:10534000EA9FF001F0E0EE83FF8331E00E948C32AF
:10535000E03011F40C94F829A0919D06A43120F4BA
:10536000A0919E06A33008F041C0E0919D06A3E005
:10537000EA9FF001EB5DF74FDF01E0919E06F0E060
:10538000AE0FBF1F0E948C32EC93E0919D060E94ED
:105390001B2FDF01E0910003F0E00E944D33EC870A
:1053A000FD87E0910503E03029F0EC85FD853A9614
:1053B000EC87FD870E9492320E9492320E949232C4
:1053C000EC85FD850E94652D0E949232EC85FD855D
:1053D0000E94322E0E948C32EA93E0E0EA930E940F
:1053E000B919E0919D06EF5FE0939D063F5FAECF58
:1053F00006C0E93521F40E94D716E89422F8E0E0CF
:10540000E093970BE22F0E94B13560960895A0E0DB
:1054100020FCA1E0A03029F4E091FD06E270E2302A
:1054200009F010C00E949732E05DEA93BFDDE6E527
:10543000EA93BCDDE2E30E949F32ED7FE093FD063C
:10544000689420F8A0E020FCA1E0A03029F4E091CD
:10545000FD06E370E13009F020C00E949732E05D64
:10546000EA93A4DDE4E5EA93A1DDE091FA06EA938C
:105470009DDDE0911E08E295EF70EA9326D0EA9355
:1054800095DDE0911E08EF70EA931FD00E949F32D5
:10549000EE7FE093FD06689420F8A0E020FCA1E0F8
:1054A000A13049F4A0E021FCA1E0A03021F4A091BA
:1054B000FC06A03009F001C08DDDE091FC06E03073
:1054C00019F0E150E093FC060895A881AA3020F479
:1054D000E881E05D0C942A2BA881AA3020F0E881B5
:1054E000E95C0C942A2BE8E50C942A2B1A930E9471
:1054F000A9320E94AE320E9458320E94B1320E94FC
:10550000A9320E940C2EE4E1F0E00E9458320E9481
:10551000B132E2EDF0E0FA93EA930E94AE320E94DB
:1055200058320E94B132E2EDF0E0FA93EA930E9421
:105530000C2EE4E1F0E00E9458320E94B132E4E126
:10554000F0E0FA93EA930E94A932E8ECF0E0FA93D3
:10555000EA93ECE3F0E00E94B7320E94AE320E9480
:1055600058320E94BD32E2EDF0E00E9458320E94B3
:1055700058320E94BD32EFE0E0930303E2E0E09393
:105580000003E0930103E5E5F0E0FA93EA93EEE12E
:10559000F0E00E94322EECEEF3E20E94762D0E94A3
:1055A0006B2DE0E0E093030319910895EEE5F1E23D
:1055B000FA93EA93EAEBEA93EAEFF0E0FA93EA93DC
:1055C000E4E0EA93E6E2EA93EEE0EA930E94B3268F
:1055D000E6EFF1E2FA93EA93EAEAEA93E7E0F1E030
:1055E000FA93EA93E8E0EA93E2E3EA93E1E0EA93EC
:1055F0000E94B3260895E991F991A991B991CD013D
:1056000061916D936623E1F7FC010895E991F991A9
:10561000A991B991CD0105900D920020E1F7FC010F
:105620000895A991B991EE27FF276D91662311F096
:105630003196FBCF0895AA27BB27E991F9910590F0
:10564000002011F01196FBCFFD0108955D9BFECF68
:10565000E881ECB9219608951A930A93AC81BD8133
:105660000E94DD333097C1F0AA81BB810E94DD33F7
:105670008F01309749F00230E0E01E0760F0F8013A
:1056800031978F01ED93FC93AC81BD810E94E12D98
:105690003197AE81A08303C0EE81EA93D7DF1981F1
:1056A0000881279608952C970E94AA3510E0E88D6E
:1056B000F98D3196E88FF98F3197E4912E2FE030F4
:1056C00011F40C940F2DE12FE03039F4253211F450
:1056D00011E002C00E94C232A1C1E130C1F4253202
:1056E00019F40E94C23299C112E0E0E0E98B00E0B7
:1056F0002D3211F401E092C12B3219F4EBE2E98B67
:105700008DC1203219F4E0E2E98B88C102C0E23099
:1057100039F450E013E0203311F400687FC102C077
:10572000E330A1F4203310F02A3308F009C0A52F8C
:10573000EAE0EA9FF0015E2FE22FE0535E0F6EC1B8
:1057400040E02E3211F414E069C110C0E430A1F43D
:10575000203310F02A3308F009C0A42FEAE0EA9FB2
:10576000F0014E2FE22FE0534E0F58C12C3619F4A2
:10577000026015E053C104C0E53011F00C940E2D09
:10578000E22FE33649F40E94CD32EE89FF89A481ED
:10579000AA930E94D33241C1E33741F40E94CD3233
:1057A0000E94DD320E94112B1E2F0AC0E037A1F4A7
:1057B0000E94CD320E94DD320E941B2B1E2F0860FA
:1057C0000F77403011F0411708F001C0142F40E06E
:1057D000E0E0E88B30E078C0E43611F0E93611F40F
:1057E000046002C0E537A1F4EAE0E88B01FF08C0DD
:1057F000E0E0FAEC6AE97BE30E94F32D1AE023C0B3
:10580000E0E1F7E260E070E00E94F32D15E01BC0DC
:10581000E83511F4086004C0E83711F00C940D2D40
:10582000E0E1E88B01FF08C0E0E0F0E060E070E15B
:105830000E94F32D18E007C0E0E0F0E160E070E0C6
:105840000E94F32D14E0403011F00F7701C041E0C9
:1058500001FF08C00E94CD32AE89BF8914960E9414
:10586000E13315C002FF0AC00E94CD32AE89BF8964
:1058700014960E94DD330E941A3309C00E94CD3273
:10588000AE89BF8914960E94DD3366277727EC879F
:10589000FD876E877F8702FF16C0AF85AA2362F45B
:1058A000EC85FD856E857F850E940433EC87FD873E
:1058B0006E877F87EDE2E98BE989E03019F01F5FA1
:1058C0004F5F01C00B7F342F00FD14C0151710F47B
:1058D000351708F00FC007FF08C002FF04C00B7F98
:1058E0002989115001C020E301C020E20E94C23288
:1058F0005150ECCF1417B0F4006102FF0AC00B7FC7
:10590000E989EA930E94D332503009F05150115086
:105910004150E0E3EA930E94D332503009F05150F5
:105920004150E8CF312FE889E030D1F43030B9F080
:1059300003FF08C0EE81FF813196EE83FF8331972C
:10594000E49105C0AE81BF81ED91AE83BF83EA9340
:105950000E94D332503009F051503150E7CF53C03C
:105960000E94E7320E947D332E2F2A3030F003FF51
:1059700002C0295C01C0295A01C0205D04FD23C07A
:10598000213350F40E94F82DA130E0E0BE07E0E0A2
:105990008E07E0E09E0709F40BC0431740F453174D
:1059A00010F000FF01C014C020E207FF0CC020E38C
:1059B000006102FF08C00B7FE989EA930E94D3329D
:1059C000503009F051500E94C232503009F051500D
:1059D00031500E94E7320E94B833EC87FD876E8712
:1059E0007F87E8890E94F82DFF27662777270E9486
:1059F0007D330E94F32DE885F9856A857B850E94B9
:105A0000A23509F0ADCF00FF08C0503031F0515041
:105A1000E0E2EA930E94D332F8CF10E048CE0E9431
:105A2000B1356A960895FF92F82E22971A930A9339
:105A3000DE010E94FC328D01DE0116960E94FC32CE
:105A40000E94DD33EA83FB83DE0114960E94FC3260
:105A50000E94DD33FA93EA931A930A930E94E62E8A
:105A60000E945B2D20DEAA81BB81E0E0EC931981CE
:105A700008812496FF900895A991B991EE270024FA
:105A800060E8E894162E169407941E2A1EF0A015BE
:105A9000B10518F0A019B109E62BB7FBAA0FBB1F7F
:105AA000669580F70895E991F99130971AF4E09599
:105AB000F09531960895E0E0F0E0FA93EA930895C6
:105AC000E091FF03F09100040895FA93EA93EFE068
:105AD000EA930C947626E1E0E0930003E09301035F
:105AE0000895E6E0F0E0FA93EA930895FA93EA93D2
:105AF0000C941417E7E0F0E0FA93EA930895A8E015
:105B0000B0E00E9401340895E0918D06F0918E0678
:105B10000895E0918906F0918A060895EAE0E093FD
:105B20006100E5E0E09362000895EA930E946D123F
:105B3000E0939B06F0939C060895E093620088EC46
:105B400090E00197F1F70895E093610088EC90E010
:105B50000197F1F70895AE0FBF1FE3E0F0E00E9458
:105B600078330895FA93EA931A930A930C9478126F
:105B7000FA93EA933A932A930C947812A09191069F
:105B8000B09192060895A0919306B091940608955D
:105B9000A5E8B6E0ED91FD913196FE93EE93089560
:105BA000A0918506B09186060895E0937906F0935A
:105BB0007A060895E0E0F0E0E0938506F09386062B
:105BC0000895ED91FD913196FE93EE930895A0E036
:105BD000B0E00E94FD3308950E94F633EA1BFB0BF0
:105BE0000E941A330895E887F9876A877B870895AA
:105BF000A885B9858A859B850895A2E0B0E00E94BA
:105C0000FD330895A4E0B0E00E94FD330895A6E0BE
:105C1000B0E00E94FD330895E2E3F0E0FA93EA93E6
:105C20000895FA93EA930C94F032A0918106B09112
:105C300082060895E0EAF0E0FA93EA930895EA9381
:105C40000E94101AE1E0E09300030895EAE0EA936D
:105C50000E94A416E0919106F091920608950E9488
:105C60000D34DACFFA93EA930C94331AFA93EA9349
:105C70000C94F416E8E1F0E0FA93EA93E8E2F0E03D
:105C800024CFE7EDF0E0FA93EA93D4CFE2E0E0939B
:105C90000003E9E6F0E0FA93EA930895EAE0EA9374
:105CA0000E94A416E0919306F091940608950A923A
:105CB0001A92FA926A937A938A939A93AA93BA93CE
:105CC000EA93FA93EFB7EA930895ACE01A9FF001D4
:105CD000E45FFC4FE0810895ACE01A9FF001EB5EB9
:105CE000FC4F08951A93E1E0EA930C94AA1AEAE0B3
:105CF000F0E097CFE093E006F093E1060895A981E4
:105D0000BA81EE27A10FBE1FEC910895FE01FA9310
:105D1000EA9308950E94EB3384E00E94132D2896A5
:105D2000F5CFF801AA81BB81EA0FFB1FE49108952A
:105D3000E091E306A6EEB6E0F0E0EE0FFF1F089557
:105D4000E091E206A6EEB6E0F0E0EE0FFF1FEA0FEC
:105D5000FB1F0895E981ACE0EA9FF0010895EF731D
:105D6000A9E2EA9FF001E757FB4F0895EF73ABE01C
:105D7000EA9FF001EB5FFB4F0895ACE01A9FF00142
:105D8000E15FFC4F0895ACE01A9FF001E35FFC4F28
:105D9000DF010E94DD330895ACE01A9FF001E35F5C
:105DA000FC4F608171811A9FF001EF5EFC4FE08132
:105DB000DB01F0E00895A083ACE01A9FF0010895A4
:105DC000ACE01A9FF001EA5EFC4F0895FE013696A2
:105DD000FA93EA930895FA93EA930C94FB2AA9E2C2
:105DE0000A9FF001E757FB4FE081E0300895A9E2F8
:105DF0000A9FF001E757FB4FFA93EA93FE013896AA
:105E0000EACFABE00A9FF001EB5FFB4FE081E030AF
:105E10000895E091E006F091E1060895A0EEB6E065
:105E2000ED91FD913296FE93EE930895E081F0E0BE
:105E3000E60FF71F0895F0E0ACE0B0E00E944D33AC
:105E400008951A930A933A932A930895E0910103CF
:105E5000F0E00895FA93EA93ED81EA93ED81EA93F5
:105E60000895E0910003ACE0EA9FF0010895F0E0AE
:105E7000EA0FFB1F0895E0930703F09308030895CA
:105E80001A93E1E0E0930103E093000310E008952A
:105E9000EF81F885EA1BFB0B0895FE01EB5BFF4FDA
:105EA000E081ACE0EA9FF001EA5EFC4FE0810895FA
:105EB000FE01EB5BFF4FE081ACE0EA9FF00108954B
:105EC000ECE8F0E00E94E7330895DE01A05CBF4FEC
:105ED000ED93FC930895FE01E85BFF4F0190F08184
:105EE000E02D0895FA01E00FF11FFA93EA93089567
:105EF000FE01EE5BFF4FE081EA930C9494261A9327
:105F00000A93FE01EC5BFF4F0190F081E02DE20F60
:105F1000F31F0895FA93EA93E5CFDDDFE20FF31F55
:105F2000FA93EA93E5CFFE01EE5BFF4FE081EA933F
:105F30000C947626FA93EA933A932A930895E5E02F
:105F4000F0E0FA93EA93C7DFFA93EA93ECCFFA937F
:105F5000EA935A934A930895DE01AC5BBF4FAC912C
:105F60000895DA01F0E00895DF01FE01EE5BFF4FD6
:105F70000190F081E02DAE17BF070895FE01EE5BA2
:105F8000FF4F0190F081E02D0895E2E0F0E00E94E3
:105F9000783308959ADFDE01AF5BBF4FAC91AA233F
:105FA0000895ECE0EA9FF001A0910003EA9FF00160
:105FB0000895AE1BBF0BE9CFECADF0E0E00FF11F91
:105FC00008953196FA93EA93D9DFE20FF31F3196E1
:105FD00049CEFA93EA93D2DFE20FF31F43CEEFAD3F
:105FE000F0E0DE011696AE0FBF1FEC910895EA9324
:105FF000EBADEA930E94B919EFADEF5FEFAF0895F3
:10600000F0E0DE011696AE0FBF1FAC9108950E941E
:106010004D33E20FF31FDF01B1DFEE0FFF1FEA0F79
:10602000FB1F08950E944D330E941A330E948C3446
:106030000895E98DFA8DE21BF30BFA93EA93089524
:10604000FA93EA93F901AD8DBE8DEA0FFB1FFA9327
:10605000EA930895FA93EA93EA8DEA930C949426CE
:10606000EBE1E0936500E4E6F0E0DBCDFA93EA9340
:106070000C940B1EEA93E1E0F0E0F8CFE3E0EA9342
:10608000E0E3F0E1F3CFE4E0EA9315CDEA93E7E053
:10609000F7E0ECCF0E940B1EE1E5EA93EFEEF0E0B3
:1060A000E5CF0E940B1EE3E5EA93EFE3F1E0DECFDC
:1060B0000E94AA35EE81AEEDB0E2F0E0EE0FFF1FD8
:1060C000EA0FFB1F0E94E7338F010895E985FA85E7
:1060D000AD85BE850895AD85BE85EFEEF0E0EA1B87
:1060E000FB0BE987FA870895EF81F885AB85BC85BE
:1060F0000895AB85BC85EFE3F1E0EA1BFB0BEF8372
:10610000F8870895EA93EE85FF85B0CFEA93EA8594
:10611000FB85AE85BF850895EA0FFB1FA7CFEA93E5
:10612000EC85FD85A3CFEA93E885F985AC85BD852F
:106130000895EF81F885E017F1070895EB85FC8558
:10614000AF81B885AE17BF0708950D851E85ED8513
:10615000FE85E987FA870D871E870B851C85EB85F1
:10616000FC85EF83F8870B871C870895ED85FE85F6
:10617000A985BA85AE17BF070895AD85BE85E985A7
:10618000FA85EA1BFB0B0895FA93EA930C94532DBE
:10619000AB85BC857DCEAF81B885EB85FC85EA1BE0
:1061A000FB0B0895D9010E944D330F010895D001D2
:1061B0000E947833AF01E0E2EA93FA01AE85BF8531
:1061C000ABCFE2E2EA931A930A930C940B1EEA9384
:1061D000F901AC85BD850895A985BA85ED85FE8553
:1061E000EA1BFB0B0895D0010E947833AF01E0E277
:1061F000EA930895E1E2EA93FA01AC85BD858CCF7C
:10620000AEEDB0E2F0E0EE0FFF1FEA0FFB1F0E94C1
:10621000E733EE83FF830895EC85F0E0EE0FFF1F78
:106220000E940C33E887F9873091000310E008954D
:10623000EA85F0E00E940E33DF01E32FF0E00E94D8
:106240004D33AF85B889EA0FFB1FAF01EA85A885FA
:10625000B9850DCEE0E2EA935A934A930C940B1E53
:10626000E885F0E00E940E33DF01E32FF0E00E94AA
:106270004D33AE85B0E0EA0FFB1FAF01EF85F88923
:1062800024913196EF87F88B0895FA93EA930C9452
:10629000FF21EA93E4E0F0E0F8CFE6E1EA93E8ECEE
:1062A000F0E0F3CFEA93E2E0F0E0EFCFEA93E1E051
:1062B000F0E0EBCFE8E2F0E0B4CC0E94AA35EE814A
:1062C000AEEFB0E2F0E0EE0FFF1FEA0FFB1F0E94FF
:1062D000E7338F010895E2E0EA93EE85FF850E949F
:1062E0001533D3CFAE0FBF1FFD010E941533CDCFA5
:1062F000E6E0EA93EC85FD850E941533C6CF0E9447
:10630000FF21E5E0EA93EFEEF0E0BFCFE9E0EA93AA
:10631000EFE3F1E0BACF0E941533B7CFEA93EC85F3
:10632000FD85F070B2CFE6E0EA93EE85FF85F3CF0E
:10633000E7E0EA93EE85FF85F070A7CFD0010E94D9
:106340007833AF01E2E0EA93FA01AE85BF85CACFA8
:10635000E3E0EA93FA01AE85BF85AE0FBF1FEFEF12
:10636000F0E0EA23FB2391CFA21BB30BEFEFF0E0A9
:10637000EA23FB238ACFE2E2EA931A930A930C946E
:10638000FF21AE0FBF1FEFEFF0E0EA23FB237DCF2D
:10639000D0010E947833AF01E2E0EA930895E6E08D
:1063A000EA93FA01AC85BD859DCFE7E0EA93FA0157
:1063B000AC85BD85E6CFAEEFB0E2F0E0EE0FFF1F9B
:1063C000EA0FFB1F0E94E733EE83FF830895E3E0AB
:1063D000EA93FA01F07059CFEF81F885FA93EA93C6
:1063E0000895EE81FF81FA93EA93EF81EA9308958D
:1063F000EC81FD81FA93EA93EC81FD812BCDAA9388
:10640000EA93FA93EFB7EA930895E0918B0AF0913B
:106410008C0A0895ABE8BAE0D4CBE0E0F0E0E0937A
:106420008B0AF0938C0A0895F0DFE550F74F008354
:10643000F1CFE0918D0AF0918E0A0895A0918B0A18
:10644000B0918C0AEA17FB070895E091960BF0E0F3
:10645000EB56F54FE081E0939C00E091960BEF5FE7
:10646000E093960B0895F0E0E030A1E0FA0708957C
:10647000E091980BF0E0E756F44F0895E32FE150D8
:10648000A8E9B0E0F0E0EE0FFF1FEA0FFB1F0E944B
:10649000E733FA93EA93E32FA8E9B0E0F0E0EE0FD8
:1064A000FF1FEA0FFB1F0E94E733FA93EA93089558
:1064B000FA93EA93E4E1F0E00895F0E0EE0FFF1FB5
:1064C000EA0FFB1F0E94E7333396AF010895E02FD8
:1064D000AEE1B1E2F0E00E941033EA0FFB1F089535
:1064E000FA93EA93E0919C0BEA93E5CAEDE9FBE0AD
:1064F000FA93EA930C948517F0E0EE0FFF1FEA0F72
:10650000FB1F0E94E7333396EE87FF8720CDFA9377
:10651000EA93EAE4F0E0E4CFE32FF0E0E756F44F4B
:10652000E0810895EC85FD85FA93EA930895E0E013
:10653000E093950BE2E0EA930E94D627E0CAEA9343
:106540000E94D627E3E0EA930E94D627E091FD0659
:106550000895EAE0F0E0FA93EA930895EAE0F0E0C3
:10656000A7CFFA93EA93ECE0EA930C947E1DFA939A
:10657000EA93ECE0EA930C947626FA93EA93E8E245
:10658000F0E0F5CF2A93ED89FE89FA93EA93FE01B4
:106590007596FA93EA930C942C2BEE89FF89349725
:1065A000EE8BFF8B0895ED89FE89FA93EA93FE0145
:1065B0007596FA93EA930C942C2BAE89BF891496A6
:1065C0000E94DD33EE83FF83FA93EA930895E88512
:1065D000F9856A857B85AC85BD858E859F85089507
:1065E000E991F991309639F080EA9FE00197F1F74F
:1065F000A8953197C9F708950024AF0DB01D0895EF
:10660000F195E195F0400895F09560957095E195CC
:10661000FF4F6F4F7F4F0895EE0FFF1FEE0FFF1FCD
:10662000EE0FFF1FEE0FFF1F0895EF2FFF27E7FD6F
:10663000FFEF08956F2F660F660B762F0895EA1708
:10664000FB07E1E00CF0EE270895FA9FF02DEB9F99
:10665000F00DEA9FE02DF10D08957A9F702D6B9F4C
:10666000700DF89F700DE99F700D6A9F602D710D80
:10667000FB9F600D711DE89F600D711D8827FA9FBB
:10668000F02D610D781FEB9FF00D611D781FEA9FC3
:10669000E02DF10D681F781F08956ED0D6DF0EF43F
:1066A000AFDF089577D0D9DF0EF4AEDF0895002470
:1066B00098E0AA0F001C0E1A10F40E0E01C0A16083
:1066C0009A95B9F7EA2FA02D08950024112490E19E
:1066D000AA0FBB1F001C111C0E1A1F0A18F40E0E65
:1066E0001F1E01C0A1609A9599F7FD01D001089580
:1066F00043D0EBDF0EF484DF08953F934F935F9315
:10670000002411244427552730E2AA0FBB1F881FFD
:10671000991F001C111C441F551F0E1A1F0A460BFF
:10672000570B28F40E0E1F1E461F571F01C0A160F5
:106730003A9559F7FD01BC01D001CA015F914F9113
:106740003F91089527D0D9DF0EF45EDF0895AFDFC3
:10675000EA2F0895E894B7FF04C0A095B09511966C
:106760006894F7FD4DDFB1DFFD010EF449DF0895B8
:10677000C4DFFD01BC010895E894F7FF02C040DFCB
:106780006894B7FF06C0A095B095119600F80394E1
:1067900000FA0895E89477FF02C036DF689497FF07
:1067A0000BC00024A095B095809590951196801D02
:1067B000901D00F8039400FA0895ED91FC91119753
:1067C0000895ED91FD916D917C9113970895059039
:1067D000F491E02D08957A936A93FA93EA930895D9
:1067E000182E862F612D192E972F712D1B2EBF2F3E
:1067F000F12D1A2EAE2FE12D0895119602D0FE2F05
:106800001197E199FECFFF93FFB7F894AEBBBFBBE2
:10681000E09AEDB3FFBFFF91089507D01196EF9373
:10682000EF2F03D0EF9111970895E19B02C0A89537
:10683000FCCF9FB7F894AEBBBFBBE09A8DB3E8170F
:1068400019F0EDBBE29AE19A9FBF0895552342F4F7
:10685000503811F4E0FF04C03196691F791F6BF0C6
:1068600050E8572711F45F93C8C05F3F31F0660FBF
:10687000000C57956795752F08955F9300200AF0D7
:10688000C8C0C1C050E8192E1522880F991F95273E
:10689000550F879550E8072E0522660F771F75273D
:1068A000550F67950895689401C0E8945F93F2DFEF
:1068B000703818F07F3F08F4A0C056E1571BAAF4C7
:1068C000519558300EF4593030F0EFEFFFEF6FEF85
:1068D0007FE777F91AC077275523B9F0EE0FFF1F2E
:1068E000661F771F5A95D1F710C07727583028F0C8
:1068F000EF2FF62F672F5850F9CF552331F07695AB
:106900006795F795E7955A95D1F700200AF47CDE54
:106910005F910895689401C0E8943097604070409A
:10692000B1F0002426F0772312F400946DDE172EC8
:106930007EE1112032F07A95EE0FFF1F661F111CC9
:10694000F9CFEF2FF62F612D5F938ADF5F910895C6
:106950004F93AF01FD01DA01AB01BC01CA01402D2B
:10696000012C142E4F910895EA0FFB1F681F089504
:10697000E095F0956095EF5FFF4F6F4F08955F933F
:1069800081DF903849F150E81526703821F1572FF2
:10699000591B13F112F4DCDFFACF583118F0AA2793
:1069A000BB278827583028F0AB2FB82F882758509E
:1069B000F9CF552329F08695B795A7955A95D9F71C
:1069C000502D512562F0D0DF38F46795F795E795A3
:1069D000739513F41EC0BCDF43DF5F910895EA1B7B
:1069E000FB0B680B51F010F40094C2DF6623A2F396
:1069F000EE0FFF1F661F7A95CBF7EE27FF2766275E
:106A000077275F910895EFEFFFEF6FE77FEF5F91DB
:106A10000895EFEFFFEF6FE77FE75F9108955F93D2
:106A200031DF703851F3903841F301240894791F15
:106A300023F41CF300203AF3ECCF0F921F932F9313
:106A40003F934F93112722279927689FA0018F9F7B
:106A5000302D410D591F6B9F300D411D591F8E9FC9
:106A600027D0BF9F25D06A9F23D0BE9F1DD0AF9F48
:106A70001BD0AE9F110D291F391F491F591FE32F2E
:106A8000F42F652F522F4F913F912F911F910F900F
:106A900066232AF0550FEE1FFF1F661F02C0739575
:106AA0004BF2D4DE5F910895100D211D391F02C0F5
:106AB000200D311D491F591F08955F93E3DE703883
:106AC00021F411200AF49FCFA4CF903809F495CF78
:106AD00001240894970B1BF4D4F30020F3CF792FF3
:106AE0001F932F933F934F9311241127222733276E
:106AF0004427552790E2AE17BF078607410730F0BD
:106B0000AE1BBF0B860B410B089401C08894551F28
:106B1000221F331F111CAA1FBB1F881F441F9A95D9
:106B200051F7F901612D4F913F912F911F916623EC
:106B300032F0550FEE1FFF1F661F7A9543F286DE77
:106B40005F910895309760407040089500240A16C0
:106B50000B0608955A934A933A932A931A930A93E9
:106B600008955D814C813B812A81198108810895B6
:00000001FF
